:1000000051EF20F00000000033EF1FF0000000006F
:0C00100000000000000000001EEF20F0C7
:0E001C00ADB202D00000FCD7CAC4AEFF120085
:0E002A00A8B202D00000FCD7CAC4A9FF120081
:100038000B840BAE27EF00F0010E036E026A016A13
:0A004800006A0A360232FF0E1200B1
:0E005200026A016A006A086A036A000E120060
:100060000B820BAE3AEF00F003680268016800688B
:080070000A360232FF0E1200F5
:080078000AAE029E000E120008
:100080000CB082EF00F00CA228EF01F00E6A000E17
:10009000026499EF00F0F00E0214D8A464EF00F0AF
:1000A000023A01380F0B02260138F00B016E0038BE
:1000B0000F0B01260038F00B006E08380F0B0026DE
:1000C0000838F00B086E0E84D89002BE7DEF00F069
:1000D00008360036013602360E2A02BE7DEF00F0E9
:1000E00008360036013602360E2A02BE7DEF00F0D9
:1000F00008360036013602360E2A0E5003641EEF13
:1001000001F0035E0BBC08AE23EF01F0D880800E37
:1001100008640030000E002201220222D8A023EF42
:1001200001F0023201320032034A28EF01F023EFDE
:1001300001F001C002F000C001F008C000F0086A40
:10014000000E0E860264D0EF00F0F00E0214D8A468
:10015000B8EF00F0023A01380F0B02260138F00B1D
:10016000016E00380F0B01260038F00B006E0E8474
:10017000D89002BE7DEF00F00036013602360E2A1E
:1001800002BE7DEF00F00036013602360E2A02BEB6
:100190007DEF00F00036013602360E2A7DEF00F0CA
:1001A00001C002F000C001F0006A000E0E960E8839
:1001B0000264FDEF00F0F00E0214D8A4E8EF00F0A6
:1001C000023A01380F0B02260138F00B016E0E8443
:1001D000D89002BE7DEF00F0013602360E2A02BE34
:1001E0007DEF00F0013602360E2A02BE7DEF00F0F0
:1001F000013602360E2A7DEF00F001C002F0016ADE
:10020000000E0E8602642DEF01F0F00E0214D8A449
:100210000CEF01F0023A0E84D89002BE7DEF00F0A0
:1002200002360E2A02BE7DEF00F002360E2A02BE12
:100230007DEF00F002360E2A7DEF00F0010E0C6E0D
:10024000FBDE30EF01F0020E0C6E16DF30EF01F036
:10025000040E0C6E05DF30EF01F0080E0C6EF9DEB7
:0202600012008A
:1002620073B409D01F0E7114016E0150000A03E12C
:0A027200010E006E01D0006A1200B8
:10027C00F250026EF29E0500FF6A0150FE6E0050B5
:08028C00FD6E02BEF28E1200AD
:10029400220E0C6E086A096A0A6A0B6A0C06D8B444
:1002A4001FD0D8900B320A3209320832033202329C
:1002B40001320032D8A0F2D70C06D8B409D00450C9
:1002C40008260550092206500A2207500B22EAD7B5
:1002D400045008260550092206500A2207500B2212
:0202E400120006
:1002E6000050086E0150006E0250016E0350026EFF
:1002F600036A0B6A0C6A9E0E036E0A6A02AE90EFE0
:1003060001F0081E001E011E021E082AD8B4002A8B
:10031600D8B4012AD8B4022A0A8E020E0C6EADDEBB
:020326001200C3
:100328000401C451390806E3300EC45D03E3010E2D
:08033800006E01D0006A120002
:1003400049C0C6F44AC0C7F44BC0C8F44CC0C9F495
:100350000401C46BC56BC551120802E1C4518E087B
:1003600008E37FDF005201E004D00401C44BC52B39
:10037000F2D70401120EC55D02E18F0EC45D03E3E6
:100380007B0E006E24D0718071A020D049504A109D
:100390004B104C101AE0C651C711C811C9110EE11B
:1003A00072C2E1FF73C2E2FF050EE66E70C200F09A
:1003B00071C201F063DF010E006E09D0010E04016D
:1003C000C65F000EC75BC85BC95BDED7006A120060
:0E03D000550EA76EAA0EA76E0E01BF81120079
:0E03DE00550EA76EAA0EA76E0E01BF9112005B
:1003EC00A49EC4C475FF49C0C5F44AC0C6F44BC032
:1003FC00C7F44CC0C8F473A421D049504A104B1018
:10040C004C101BE00401C551C611C711C8110EE1F7
:10041C0072C2E1FF73C2E2FF040EE66E70C200F01E
:10042C0071C201F025DF010E006E3AD0010E0401FD
:10043C00C55F000EC65BC75BC85BDDD749C0C5F4A2
:10044C004AC0C6F44BC0C7F44CC0C8F4A4BE21D0FB
:10045C0049504A104B104C101BE00401C551C611F9
:10046C00C711C8110EE172C2E1FF73C2E2FF040EA4
:10047C00E66E70C200F071C201F0FADE010E006E81
:10048C000FD0010E0401C55F000EC65BC75BC85BD5
:10049C00DDD771BC02D0006A03D07184020E006EED
:0204AC0012003C
:1004AE000401C451200A09E0C4510D0804E3090EE9
:1004BE00C45D01E302D0006A02D0010E006E12008C
:1004CE00C7B409D01F0EC514016E0150000A03E116
:0A04DE00010E006E01D0006A12004A
:0404E8007184120009
:1004EC0003500718D8A48AEF02F002500618D8A4BB
:1004FC008AEF02F001500518D8A48AEF02F00050E0
:0E050C000418D8B4D8841200D894120012003B
:10051A000B800BAE99EF02F0026A0AAEFF0E026E72
:0C052A00016E006E0A360232FF0E120055
:10053600025006180E6E086A096A0B6A03500764B1
:100546008EEF03F006500A6E068E028E03500B6E77
:100556000750036E000E0B64DEEF02F00B50075ED1
:10056600D8B47FEF03F0070E07644DEF03F0075E84
:1005760000C008F001C000F002C001F0026A074E98
:100586007FEF03F0076422EF03F0075E00C008F078
:1005960001C000F0016A074E7FEF03F0076400EF29
:1005A60003F0075E00C008F0006A074E7FEF03F015
:1005B6000764E7EF02F00AC002F005C001F004C0CC
:1005C60000F0086AABEF04F0030E0764F2EF02F0E6
:1005D600075E08380F0B086E074E7FEF03F0D890C2
:1005E6000832074E7FEF03F0D8900832074E7FEFB0
:1005F60003F0D89008327FEF03F0030E076411EF83
:1006060003F0075E08380F0B086E0038F00B08265B
:1006160000380F0B006E074E7FEF03F0D8900032C4
:100626000832074E7FEF03F0D89000320832074EAB
:100636007FEF03F0D890003208327FEF03F0030E0D
:10064600076439EF03F0075E08380F0B086E0038B1
:10065600F00B082600380F0B006E0138F00B002651
:1006660001380F0B016E074E7FEF03F0D890013271
:1006760000320832074E7FEF03F0D8900132003285
:100686000832074E7FEF03F0D8900132003208326D
:100696007FEF03F0030E07646AEF03F0075E083886
:1006A6000F0B086E0038F00B082600380F0B006E93
:1006B6000138F00B002601380F0B016E0238F00BE3
:1006C600012602380F0B026E074E7FEF03F0D8901B
:1006D6000232013200320832074E7FEF03F0D89023
:1006E6000232013200320832074E7FEF03F0D89013
:1006F6000232013200320832096A000E0EAE73EF82
:1007060004F0081E001E011E021E082A00220122F5
:10071600022273EF04F00750D8A494EF03F0ABEF76
:1007260004F0096A02C00AF0028E068E0750035CC6
:10073600076ED8B466EF04F0070E076434EF04F0D2
:10074600075E0450096E0550046E0650056E066A73
:10075600074E66EF04F0070E076409EF04F0075E24
:100766000450096E0550046E056A074E66EF04F0E4
:10077600070E0764E7EF03F0075E0450096E046A8C
:10078600074E66EF04F0070E0764CEEF03F00AC0CB
:1007960002F0ABEF04F0030E0764D9EF03F0075E37
:1007A60009380F0B096E074E66EF04F0D890093230
:1007B600074E66EF04F0D8900932074E66EF04F054
:1007C600D890093266EF04F0030E0764F8EF03F0E1
:1007D600075E09380F0B096E0438F00B092604383A
:1007E6000F0B046E074E66EF04F0D8900432093200
:1007F600074E66EF04F0D89004320932074E66EFD2
:1008060004F0D8900432093266EF04F0030E076450
:1008160020EF04F0075E09380F0B096E0438F00B61
:10082600092604380F0B046E0538F00B042605382C
:100836000F0B056E074E66EF04F0D89005320432B2
:100846000932074E66EF04F0D890053204320932B9
:10085600074E66EF04F0D89005320432093266EF8F
:1008660004F0030E076451EF04F0075E09380F0B1E
:10087600096E0438F00B092604380F0B046E053890
:10088600F00B042605380F0B056E0638F00B05260F
:1008960006380F0B066E074E66EF04F0D890063248
:1008A600053204320932074E66EF04F0D89006325C
:1008B600053204320932074E66EF04F0D89006324C
:1008C600053204320932086A000E0EAE73EF04F0E8
:1008D600091E041E051E061E092A042205220622DA
:1008E6000950082604500022055001220650022213
:1008F6000EBE8AEF04F0D8A099EF04F0023201325E
:1009060000320832033E99EF04F0A5EF04F0D8B0A8
:100916009FEF04F0000E081E001E011E021E082A8C
:100926000022012202220A7E9FEF04F0010E0C6EC5
:1009360040EC00F0ADEF04F0020E0C6E40EC00F05F
:10094600ADEF04F0040E0C6E30EC00F0ADEF04F0E9
:06095600000E0C6E120001
:10095C000C6A0E6A0250D8A4C7EF04F001C002F072
:10096C0000C001F0006A0E860250D8A4C7EF04F054
:10097C0001C002F0016A0E960E880250D8B4D9EF6D
:10098C0004F00E50035ED8A4D8A0DFEF04F0D8908A
:10099C0002BEE5EF04F0003601360236032ECEEF30
:1009AC0004F0DFEF04F0010E0C6E29EC00F0E9EF1F
:1009BC0004F0020E0C6E1CEC00F0E9EF04F0040ED7
:0809CC000C6E3CEC00F012007F
:0809D4000B6A0B86FF0E1200F6
:1009DC000A6A0350D8A40A800750D8A40A820A5085
:1009EC00D8B451EF05F0030AD8B40AEF05F00AB0F9
:1009FC0005EF05F006AE4FEF05F04DEF05F002AE3A
:100A0C004DEF05F04FEF05F00250800B0A6E029E81
:100A1C000650800B069E0A18D8B41BEF05F00A503E
:100A2C00D8B44DEF05F04FEF05F00750035CD8B488
:100A3C0025EF05F0D8A041EF05F047EF05F0065083
:100A4C00025CD8B42FEF05F0D8A041EF05F047EFCA
:100A5C0005F00550015CD8B439EF05F0D8A041EF92
:100A6C0005F047EF05F00450005CD8B451EF05F0E9
:100A7C00D8B047EF05F00A52D8B44FEF05F04DEF60
:100A8C0005F00A52D8B44DEF05F04FEF05F0D880C1
:0E0A9C001200D8901200D880D88412001200E8
:100AAA00086A096A000E07620364DAEF05F0025069
:100ABA0006180A6E075003267E0ED8A06BEF05F0C3
:100ACA00035ED8B0DFEF05F06FEF05F0035ED8A044
:100ADA00E4EF05F0028E068E02C00EF001C00BF0A4
:100AEA0000C00DF000500402F4CF0CF001500502D2
:100AFA00F4CF00F0F3CF08F00402F3500C26F450C0
:100B0A000822000E00220D500502F3500C26F45064
:100B1A000822000E002202500402F3500826F45064
:100B2A00002202500502016A000E0122F35000263B
:100B3A00F45001220D500602F3500826F450002208
:100B4A00026A000E012202220B500602F35000260E
:100B5A00F4500122000E02220E500602F350012622
:100B6A00F450022202BEC2EF05F008360036013602
:100B7A0002360306D8B4E4EF05F0D5EF05F0D880C5
:100B8A00800E08640030000E002201220222D8A042
:100B9A00D5EF05F0023201320032034ADFEF05F0E9
:100BAA000AAE029E000EE7EF05F0010E29EC00F0F6
:100BBA00E7EF05F0020E30EC00F0E7EF05F0040E67
:060BCA001CEC00F012001B
:100BD000A0EC01F0780E0401C46F08DC31EC01F0E8
:100BE0000050000A01E1FAD7400E0401C46FF6EC90
:100BF00001F031EC01F00050000A01E1FAD7B9C46C
:100C0000C4F4F6EC01F063DC0050000A01E1FBD70C
:040C10006BDC120087
:100C140000C008F00150006E016A026A036A0B6AA0
:100C24000C6A016A026A036A960E036E0A6A00AECF
:100C340022EF06F0081E001E082AD8B4002A0A8EE5
:100C440000C001F008C000F0086A026A85DE1200E4
:100C5400A0EC01F0780E0401C46FF6EC01F031EC65
:100C640001F00050000A01E1FAD7800E0401C46FBC
:100C7400F6EC01F031EC01F00050000A01E1FAD782
:100C8400B9C4C4F4F6EC01F031EC01F00050000AF0
:100C940001E1FAD727DC31EC01F00050000A01E150
:040CA400FAD7120069
:100CA800086A096A100E0C6E0134083609360450B9
:100CB800085E0550D8A0053C095ED8B007D004509E
:100CC80008260550D8B0053C0926D89000360136CC
:060CD8000C2EEAD7120009
:100CDE00086A080E0C6E003408360450085ED8B050
:0E0CEE0002D00826D89000360C2EF5D7120042
:100CFC000B6A0350D8B4C4EF06F002500A6E028E91
:100D0C008E0E035E03AEC8EF06F0036C080E035C98
:100D1C00D8A0A3EF06F0036E013602C001F0026A00
:100D2C00080E035CD8A0A3EF06F0036E0136016A2F
:100D3C000350D8A4D890ADEF06F00350D8B4ADEF63
:100D4C0006F0D89002320132032EA7EF06F00BBC4E
:100D5C0001A0BAEF06F0D8A0BAEF06F0012AD8B479
:100D6C00022A02BED7EF06F00AAEDDEF06F0021E35
:100D7C00011E012AD8B4022ADDEF06F0026A016ACC
:100D8C00DDEF06F00B800BAEE1EF06F0026A0AAE67
:100D9C00E1EF06F0FF0E026E016E0A360232E1EF51
:100DAC0006F0010E0C6E8DEC02F0E3EF06F0000E77
:100DBC000C6EE3EF06F0FF0E0C6E0150006E02504D
:040DCC00016E1200A2
:100DD0000B6A0C6A086A0350D8B46CEF07F002C0C3
:100DE0000AF0028E9E0E035E03AE5CEF07F0036C0A
:100DF000080E035CD8A029EF07F0036E083600C088
:100E000008F001C000F002C001F0026A080E035CA5
:100E1000D8A029EF07F0036E083600C008F001C023
:100E200000F0016A080E035CD8A029EF07F0036EFA
:100E3000083600C008F0006A080E035CD8A029EF4D
:100E400007F0036E0836086A0350D8A4D89035EF2F
:100E500007F00350D8B435EF07F0D89002320132D2
:100E600000320832032E2DEF07F00BBC08A046EF2E
:100E700007F0D8A046EF07F0082AD8B4002AD8B463
:100E8000012AD8B4022A02BE70EF07F00AAE6CEF56
:100E900007F0021E011E001E081E082AD8B4002AF0
:100EA000D8B4012AD8B4022A6CEF07F0026A016AAA
:100EB000006A086A6CEF07F00B800BAE77EF07F063
:100EC000026A0AAE77EF07F0026E016E006E086EDE
:100ED0000A36023277EF07F00C6A000E78EF07F05F
:100EE000010E0C6E000E8DEC02F078EF07F0FF0E95
:100EF0000250036E0150026E0050016E0850006EE9
:020F00001200DD
:080F0200067E9BEC02F01200D8
:100F0A000401B951180808E3B9510D0804E2110E99
:100F1A00B95D01E201D002D0006AFAD1BA51000AE1
:100F2A00D8A48FD0BC5302E0EFEC01F042D0BBC48E
:100F3A00C0FE82D0BBC4C1FE7FD0BBC4C2FE7CD07F
:100F4A00BBC4C3FE79D0BBC4C4FE76D0BBC4C5FE45
:100F5A0073D0BBC4C6FE70D0BBC4C7FE6DD0BBC4C1
:100F6A00C8FE6AD0BBC4C9FE67D0BBC4CAFE64D07F
:100F7A00BBC4CBFE61D0BBC4CCFE5ED0BBC4CDFE2D
:100F8A005BD0BBC4D1FE58D0BBC4D2FE55D0BBC4C3
:100F9A00D3FE52D0BBC4D4FE4FD0BBC4D5FE4CD076
:100FAA00BBC4D6FE49D0BBC4D7FE46D0BBC4D8FE0C
:100FBA0043D00401B951000ABAE0B951010ABAE0B2
:100FCA00B951020ABAE0B951030ABAE0B951040A9E
:100FDA00BAE0B951050ABAE0B951060ABAE0B951FC
:100FEA00070ABAE0B951080ABAE0B951090ABAE0DF
:100FFA00B9510A0ABAE0B9510B0ABAE0B9510C0A56
:10100A00BAE0B9510D0ABAE0B951110ABAE0B951B8
:10101A00120ABAE0B951130ABAE0B951140ABAE08D
:10102A00B951150ABAE0B951160ABAE0B951170A04
:10103A00BAE0B951180ABAE00401BC5302E0E8EC7C
:10104A0001F00401BA51010AD8A477D0BC5302E0D6
:10105A00EFEC01F036D0B9C4E1FE6AD0B9C4E2FEC1
:10106A0067D0B9C4E3FE64D0B9C4E4FE61D0B9C4A0
:10107A00E6FE5ED0B9C4E7FE5BD0B9C4E8FE58D03C
:10108A00B9C4E9FE55D0B9C4EAFE52D0B9C4F2FED9
:10109A004FD0B9C4F3FE4CD0B9C4F4FE49D0B9C498
:1010AA00F7FE46D0B9C4F8FE43D0B9C4FCFE40D01E
:1010BA00B9C4FDFE3DD0B9C4FEFE3AD0B9C4FFFEA4
:1010CA0037D00401BB51000AC6E0BB51010AC6E091
:1010DA00BB51020AC6E0BB51030AC6E0BB51040A6F
:1010EA00C6E0BB51050AC6E0BB51060AC6E0BB51C1
:1010FA00070AC6E0BB51080AC6E0BB51090AC6E0A6
:10110A00BB510A0AC6E0BB510B0AC6E0BB510C0A26
:10111A00C6E0BB510D0AC6E0BB510E0AC6E0BB5180
:10112A000F0AC6E0BB51100AC6E0BB51110AC6E05D
:10113A000401BC5302E0E8EC01F09AD00401BAB110
:10114A0002D0929001D09280E1D00401BAB102D0CB
:10115A00929201D09282DAD00401BAB102D0929A64
:10116A0001D0928AD3D00401BAB102D0939001D0AF
:10117A009380CCD00401BAB102D0939201D0938269
:10118A00C5D00401BAB102D0939401D09384BED0E1
:10119A000401BAB102D0939601D09386B7D0040164
:1011AA00BAB102D0939801D09388B0D00401BAB1F1
:1011BA0002D0939A01D0938AA9D00401BAB102D07D
:1011CA00939C01D0938CA2D00401BAB102D0939E11
:1011DA0001D0938E9BD00401BAB102D0949001D071
:1011EA00948094D00401BAB102D0949201D094822E
:1011FA008DD00401BAB102D0949401D0948486D0DF
:10120A000401BAB102D0949C01D0948C7FD004011D
:10121A00BAB102D0949E01D0948E78D00401BAB1AA
:10122A0002D0959401D0958471D00401BAB102D04C
:10123A00959601D095866AD00401BAB102D09598E4
:10124A0001D0958863D00401BAB102D0959A01D031
:10125A00958A5CD00401BAB102D0959C01D0958CD4
:10126A0055D00401BAB102D0959E01D0958E4ED0C8
:10127A000401B951000AD8B461D7B951010AD8B4E6
:10128A0064D7B951020AD8B467D7B951030AD8B496
:10129A006AD7B951040AD8B46DD7B951050AD8B476
:1012AA0070D7B951060AD8B473D7B951070AD8B456
:1012BA0076D7B951080AD8B479D7B951090AD8B436
:1012CA007CD7B9510A0AD8B47FD7B9510B0A83E03F
:1012DA00B9510C0A87E0B9510D0A8BE0B951110ACC
:1012EA008FE0B951120A93E0B951130A97E0B95144
:1012FA00140A9BE0B951150A9FE0B951160AA3E0F6
:10130A00B951170AA7E0B951180AABE0FF0E006EEF
:02131A001200BF
:10131C000401BB51BC1108E0BBC4E1FFBCC4E2FF3B
:10132C00B9C4E6FFBAC4E6FFB9C4E9FFBAC4EAFF20
:10133C00EECF00F000C0BFF400C0C4F457EC02F0D4
:10134C00005203E0B94BBA2BEFD7BD6B000EBFBFF9
:10135C00FF0E006E000E001802E12D0EBF1905E104
:10136C00010EBD6FB94BBA2B0CD0000EBFBFFF0ED8
:10137C00006E000E001802E12B0EBF1902E1B94BF2
:10138C00BA2BBF6BC06BC16BC26BC36BBE6BBDB9F1
:10139C000BD0B9C4E9FFBAC4EAFFEE502E0A04E13F
:1013AC00BD89B94BBA2B59D0B9C4E9FFBAC4EAFF0D
:1013BC00EECFC4F494EC01F0005201E14FD0BD83A8
:1013CC00000EBFBFFF0E000A02E1080EBF1940E07D
:1013DC00BDA901D0BE07BF2BC0C400F0C1C401F031
:1013EC00C2C402F0C3C403F00A0E046E000E056EF4
:1013FC00066E076E4AEC01F000C0C0F401C0C1F4E7
:10140C0002C0C2F403C0C3F400000000B9C4E9FF79
:10141C00BAC4EAFF300EEE5C006E016A000E015A8F
:10142C00000E01BEFF0E026E036EC0510026C151AC
:10143C000122C2510222C351032200C0C0F401C0D8
:10144C00C1F402C0C2F403C0C3F40000000003D016
:10145C00BDB901D0BE2BB94BBA2B99D7BF6BB9C450
:10146C00E9FFBAC4EAFFEE50650A08E0B9C4E9FF27
:10147C00BAC4EAFFEE50450A01E068D0B94BBA2B6A
:10148C00B9C4E9FFBAC4EAFFEE502D0A04E1BD87E6
:10149C00B94BBA2B09D0B9C4E9FFBAC4EAFFEE5074
:1014AC002B0A02E1B94BBA2BB9C4E9FFBAC4EAFF63
:1014BC00EE50300A03E1B94BBA2BF6D7B9C4E9FFA9
:1014CC00BAC4EAFFEECFC4F494EC01F0005239E058
:1014DC00B9C4E9FFBAC4EAFF300EEE5CBF6FB94B7A
:1014EC00BA2BB9C4E9FFBAC4EAFFEECFC4F494EC4A
:1014FC0001F0005226E00A0EBF03F3CFBFF4B9C4CB
:10150C00E9FFBAC4EAFF300EEE5C006E0050BF2754
:10151C00B94BBA2BB9C4E9FFBAC4EAFFEECFC4F495
:10152C0094EC01F000520DE00A0EBF03F3CFBFF4B0
:10153C00B9C4E9FFBAC4EAFF300EEE5C006E00508D
:10154C00BF27BDA703D0BF510008BF6FBF51BE2737
:10155C00000EBC1902E1000EBB190AE0BDA308D0B5
:10156C00BBC4E1FFBCC4E2FFB9C4E6FFBAC4E6FFEA
:10157C00C0C400F0C1C401F0C2C402F0C3C403F083
:10158C0073EC01F000C0C0F401C0C1F402C0C2F49D
:10159C0003C0C3F4046A056A066A076AC0C400F093
:1015AC00C1C401F0C2C402F0C3C403F076EC02F073
:1015BC00010ED8A4000E006E005205E0006A016A0C
:1015CC00026A036A04D1800EBE19006E800E000AF6
:1015DC00005CD8B073D0BE510008BE6F800EBE192F
:1015EC00006E800E0A0A005C1DE3C0C400F0C1C48A
:1015FC0001F0C2C402F0C3C403F0FF0E046EE60E89
:10160C00056E5B0E066E5D0E076E55EC05F000C0A8
:10161C00C0F401C0C1F402C0C2F403C0C3F40A0E8A
:10162C00BE5FDCD7BE51000A1CE0C0C400F0C1C4D0
:10163C0001F0C2C402F0C3C403F0CD0E046ECC0E94
:10164C00056E4C0E066E7B0E076E55EC05F000C059
:10165C00C0F401C0C1F402C0C2F403C0C3F4BE079D
:10166C00E1D7010E046E000E056E000E066E010E23
:10167C00076EC0C400F0C1C401F0C2C402F0C3C400
:10168C0003F0EEEC04F0010ED8B0000E006E005228
:10169C0014E0BDA109D0010E006E000E016E800E8B
:1016AC00026E030E036E93D0010E006E000E016EDF
:1016BC00000E026E010E036E8AD072D0800E000AEC
:1016CC00006E800EBE19005C6BE20A0EBE5D1DE35F
:1016DC00C0C400F0C1C401F0C2C402F0C3C403F022
:1016EC00F90E046E020E056E150E066EA00E076E38
:1016FC0055EC05F000C0C0F401C0C1F402C0C2F446
:10170C0003C0C3F40A0EBE5FE0D7BE51000A1CE052
:10171C00C0C400F0C1C401F0C2C402F0C3C403F0E1
:10172C00000E046E000E056E200E066E820E076E05
:10173C0055EC05F000C0C0F401C0C1F402C0C2F405
:10174C0003C0C3F4BE07E1D7C0C404F0C1C405F0A4
:10175C00C2C406F0C3C407F0FF0E006EFF0E016E8C
:10176C007F0E026EFF0E036EEEEC04F0010ED8B08D
:10177C00000E006E005214E0BDA109D0FF0E006EE9
:10178C00FF0E016EFF0E026EFF0E036E20D0FF0ED9
:10179C00006EFF0E016E7F0E026EFF0E036E17D0F1
:1017AC00BDA10DD0000EC019006E000EC119016E46
:1017BC00800EC219026E000EC319036E08D0C0C48D
:1017CC0000F0C1C401F0C2C402F0C3C403F01200A3
:1017DC000B6A0A6A096A00500402F4CF09F0F3CFCD
:1017EC0008F001500502F4CF0BF0F3CF0AF00050D3
:1017FC000502F3500926F4500A22E86A0B22015024
:10180C000402F3500926F4500A22E86A0B2208C09D
:10181C0000F009C001F00AC002F00BC003F0120086
:10182C000450000A12E10550000A0FE10650000AAC
:10183C000CE10750000A09E1FF0E006EFF0E016E6D
:10184C007F0E026EFF0E036EA8D0086A096A07505D
:10185C00D8B4C1EF0CF00350D8B4C6EF0CF0025062
:10186C0006180A6E028E068E0E6A02C008F001C0BF
:10187C000CF000C00DF004500D5E0550D8A0053CD6
:10188C000C5E0650D8A0063C085E086A0C6A0D6A0D
:10189C00D8A058EF0CF0D890023201320032083246
:1018AC00010E0E6E0750035ED8A065EF0CF07E0E95
:1018BC000E240326D8B0CBEF0CF06BEF0CF07E0EA1
:1018CC000E240326D8A0D0EF0CF0180E0B6E0D369C
:1018DC000C3608360036013602360E360450005EE1
:1018EC000550D8A0053C015E0650D8A0063C025E0F
:1018FC0006340E120EA086EF0CF00D8091EF0CF05A
:10190C00045000260550D8B0053C01260650D8B02E
:10191C00062802260D900B2E6DEF0CF0B7EF0CF095
:10192C00D8900036013602360E360450005E055053
:10193C00D8A0053C015E0650D8A0063C025E0634D9
:10194C000E10010B0D26D8B00C2AD8B4082AD8A436
:10195C00B7EF0CF008320C320D32032AD8B4CBEFAF
:10196C000CF00AAE089E0850026E0C50016E0D5021
:10197C00006ED3EF0CF0010EEAEC04F0D3EF0CF098
:10198C00020E29EC00F0D3EF0CF0040E30EC00F05A
:0C199C00D3EF0CF0080E1CEC00F0120061
:1019A8000401A851000805E3070EA96F000EAA6FED
:1019B80012D0A851160805E2170EAB6F000EAC6FD7
:1019C80006D0A851010FAB6FAC6B000EAC23ABC4B3
:1019D800A9F4ACC4AAF4A9C4B3F4AAC4B4F4AD6B12
:1019E800AE6B046A056A066A076AA2C400F0A3C45B
:1019F80001F0A4C402F0A5C403F0EEEC04F0010E5B
:101A0800D8B0000E006E005209E0A6C4E1FFA7C4DA
:101A1800E2FF2D0EE66EA64BA72BA47FA2C404F00E
:101A2800A3C405F0A4C406F0A5C407F0006A016ABF
:101A3800026A036AEEEC04F0010ED8B0000E006EE4
:101A4800005237E0000E046E000E056E000E066EA2
:101A58007F0E076EA2C400F0A3C401F0A4C402F074
:101A6800A5C403F0EEEC04F0010ED8B0000E006E31
:101A780000521FE0A2C400F0A3C401F0A4C402F005
:101A8800A5C403F0000E046E000E056E200E066E4F
:101A9800820E076E55EC05F000C0A2F401C0A3F455
:101AA80002C0A4F403C0A5F4010EAD5F000EAE5B46
:101AB800C9D7000E046E000E056E200E066E820E4B
:101AC800076EA2C400F0A3C401F0A4C402F0A5C428
:101AD80003F0EEEC04F0000ED8B0010E006E0052D8
:101AE8001DE0000E046E000E056E200E066E820EBE
:101AF800076EA2C400F0A3C401F0A4C402F0A5C4F8
:101B080003F090DE00C0A2F401C0A3F402C0A4F464
:101B180003C0A5F40401AD4BAE2BCBD7AD51B32711
:101B2800AE51B423010EAF6F000EB06F000EB56F4B
:101B3800000EB66F000EB76F7F0EB86F800EB0192B
:101B4800006E800EB419005C02E1B351AF5D1DE276
:101B5800000E046E000E056E200E066E820E076ED5
:101B6800B5C400F0B6C401F0B7C402F0B8C403F0BD
:101B780059DE00C0B5F401C0B6F402C0B7F403C022
:101B8800B8F40401AF4BB02BD9D7000E046E000E89
:101B9800056E000E066E800E076EB5C400F0B6C462
:101BA80001F0B7C402F0B8C403F03CDEA2C404F0EC
:101BB800A3C405F0A4C406F0A5C407F09BEC02F08A
:101BC80000C0A2F401C0A3F402C0A4F403C0A5F4A9
:101BD800000E046E000E056E200E066E820E076E55
:101BE800EEEC04F0000ED8B0010E006E00520BE0CF
:101BF800000E0401A26F000EA36F000EA46F7F0EEB
:101C0800A56FAD4BAE2B0401800EAE19006E800E91
:101C1800005C02E1000EAD5D38E2A6C4E1FFA7C496
:101C2800E2FF300EE66EA64BA72BA6C4E1FFA7C4C1
:101C3800E2FF2E0EE66EA64BA72B800EB419006E9F
:101C4800800E005C02E1000EB35D04E2B351AD5FAB
:101C5800B451AE5BFF0EAF6FFF0EB06F800EAE19C2
:101C6800006E800EB019005C02E1AF51AD5D0DE26F
:101C7800A6C4E1FFA7C4E2FF300EE66EA64BA72B71
:101C8800010EAF5F000EB05BE9D7AF6BB06B800E93
:101C9800B019006E800EB419005C02E1B351AF5D5B
:101CA80063E2A2C400F0A3C401F0A4C402F0A5C476
:101CB80003F07EEC06F000C0B1F401C0B2F4300EBF
:101CC8000026A6C4E1FFA7C4E2FF00C0E6FFA64BBA
:101CD800A72BB051AE1902E1AD51AF1908E1A6C466
:101CE800E1FFA7C4E2FF2E0EE66EA64BA72BB1C4F8
:101CF80000F0B2C401F00AEC06F000C0B5F401C06F
:101D0800B6F402C0B7F403C0B8F400C004F001C0D0
:101D180005F002C006F003C007F0A2C400F0A3C497
:101D280001F0A4C402F0A5C403F081EC07F000C0E0
:101D3800A2F401C0A3F402C0A4F403C0A5F4000EE9
:101D4800046E000E056E200E066E820E076E55ECB0
:101D580005F000C0A2F401C0A3F402C0A4F403C0BB
:101D6800A5F4AF4BB02B93D7A6C4E1FFA7C4E2FFFD
:041D7800E66A120005
:101D7C00A2C402F0A3C403F002C000F003C001F03F
:101D8C00024A032A00C0E9FF01C0EAFFEE5201E05B
:101D9C00F3D70401A251025C006EA3510358016EEB
:0A1DAC00010E005E000E015A120045
:101DB600AFCF01F0ACA202D0AC98AC8801C000F065
:021DC600120009
:101DC800840ED56E6D0ED76E840ED66E02016093AA
:081DD800D08EF294F28A120091
:101DE0000401A66B050EA65D0AE2A651A425E16ECC
:101DF000000EA521E26E200EE66EA62BF3D7A651AB
:101E0000A425E16E000EA521E26EE66AA607A651A2
:101E1000A425A76F000EA521A86F0A0E046E000E60
:101E2000056EA2C400F0A3C401F054EC06F008C093
:101E300000F009C001F0300E0026A7C4E1FFA8C4DD
:101E4000E2FF00C0E6FF0A0E046E000E056EA2C49B
:101E500000F0A3C401F054EC06F000C0A2F401C0ED
:101E6000A3F4000E011802E1000E001801E102D0F7
:061E7000A607CDD7120009
:101E7600A6C400F00401A607005228E0A2C4E9FFA8
:101E8600A3C4EAFFEE50000A0CE0A2C4E9FFA3C413
:101E9600EAFFA4C4D9FFA5C4DAFFEE50DE1801E1BB
:101EA6000FD0A2C4E9FFA3C4EAFFA4C4D9FFA5C406
:101EB600DAFFDE50EE5C006E016A000E015A08D0B1
:101EC6000401A24BA32BA44BA52BD2D7006A016A0F
:021ED6001200F8
:0A1ED800000E9EBA010E006E12000B
:101EE200A2C4B9F4A3C4BAF40401BB6BBC6B8EECFC
:041EF20009F01200E1
:101EF6000401A46BA56BA2C403F0A3C404F0A2C49E
:101F060005F0A3C406F003C0E9FF04C0EAFFEE50E3
:101F1600200A04E1A451A51101E110D0010EA46F1D
:101F2600000EA56F03C0E9FF04C0EAFF05C0E1FF8C
:101F360006C0E2FFEECFE6FF054A062A03C001F01F
:101F460004C002F0034A042A01C0E9FF02C0EAFF06
:101F5600EE50000AD8E1A2C400F0A3C401F01200BA
:101F6600A5C400F0016A026A036AFF0E0016000E9D
:101F7600011600C0AAF401C0ABF47F0E005C026E2D
:101F8600000E0158036E02C0AAF403C0ABF4800E23
:101F96000318006E800E005C02E1000E025C22E275
:101FA600046A056A066A076AA2C400F0A3C401F0BF
:101FB600A4C402F0A5C403F0EEEC04F0010ED8B000
:101FC600000E006E005209E0000E006E000E016E5B
:101FD600800E026E7F0E036E5CD0006A016A026A92
:101FE600036A57D00401AB51000802E1AA51180850
:101FF60009E2A2C400F0A3C401F0A4C402F0A5C47F
:1020060003F047D0A2C400F0A3C401F0A4C402F0B8
:10201600A5C403F0E8EC06F073EC01F000C0A6F4EA
:1020260001C0A7F402C0A8F403C0A9F400C004F0DC
:1020360001C005F002C006F003C007F0A2C400F01C
:10204600A3C401F0A4C402F0A5C403F0EEEC04F0AE
:10205600010ED8B0000E006E005213E0000E046EA2
:10206600000E056E000E066E7F0E076EA6C400F00B
:10207600A7C401F0A8C402F0A9C403F081EC07F0DC
:1020860008D0A6C400F0A7C401F0A8C402F0A9C4F1
:0420960003F0120041
:10209A00200E0401B96F2AEC06F00401B96B2AEC90
:1020AA0006F0210E0401B96F2AEC06F0A2C4B9F4B5
:1020BA002AEC06F00401A2510F0FB96F2AEC06F0C0
:1020CA00220E0401B96F2AEC06F0010E0401B96F61
:1020DA002AEC06F0030E0401B96F2AEC06F004019B
:1020EA00A46BA56B800EA519006E800E005C02E140
:1020FA00300EA45D24E2030E006E000E016EA3C42E
:10210A0004F0000E056EEEEC0BF0280E0024E96ECA
:10211A00000E0120EA6EA451EE24F66EA551EE20BF
:10212A00F76E000EA5BFFF0EEE20F86E0900F5CF80
:10213A00B9F4E8EC05F00401A44BA52BD3D712009F
:10214A000401A56B030EA55D0AE2A551A325E16E64
:10215A00000EA421E26E200EE66EA52BF3D7A55140
:10216A00A325E16E000EA421E26EE66AA507A55139
:10217A00A325A66F000EA421A76F0A0E046EA2C49F
:10218A0000F06FEC06F008C000F0300E0026A6C47E
:10219A00E1FFA7C4E2FF00C0E6FF0A0E046EA2C474
:1021AA0000F06FEC06F000C0A2F40050000A01E152
:0821BA0002D0A507DCD71200DA
:0E21C200030E0D6E0D2EFED700000000120061
:1021D000A2C404F0A3C405F004C0E9FF05C0EAFFEF
:1021E000EE5203E0044A052AF7D704C002F005C006
:1021F00003F0044A052AA4C400F0A5C401F00401B8
:10220000A44BA52B00C0E9FF01C0EAFF02C0E1FF1B
:1022100003C0E2FFEECFE6FF02C0E9FF03C0EAFF22
:10222000EE5201E0E2D7A2C400F0A3C401F0120014
:102230000401A351B00FB96F2AEC06F00F0E040190
:10224000A215B96F2AEC06F0F00E0401A215B96FC1
:10225000B933B99FB933B99FB933B99FB933B99F6E
:08226000B9892AEC06F0120016
:102268000D0E0401CA6F15EC00F00A0E0401CA6FC6
:0622780015EC00F012005D
:0E227E00C70E0D6E0D2EFED7000000001200E0
:10228C000401A56BA2C4E9FFA3C4EAFFEECFA4F43A
:10229C00A451000A0FE0A4C4CAF415EC00F0040128
:1022AC00A52BA551A225E96E000EA321EA6EEECF57
:0622BC00A4F4EED71200AD
:1022C200A2C4B9F4A3C4BAF4A4C4BBF40401BC6BA1
:0622D20085EC07F012008C
:1022D800A2C404F0A3C405F004C002F005C003F0D2
:1022E800044A052AA4C400F0A5C401F00401A44BC3
:1022F800A52B00C0E9FF01C0EAFF02C0E1FF03C04F
:10230800E2FFEECFE6FF02C0E9FF03C0EAFFEE52AC
:0E23180001E0E2D7A2C400F0A3C401F012005D
:10232600A2C4E9FFA3C4EAFFEE500401A41905E123
:10233600A2C400F0A3C401F010D0A2C400F0A3C44C
:1023460001F0A24BA32B00C0E9FF01C0EAFFEECFCC
:0C23560000F00052E5E1006A016A12008C
:10236200080E0C6EC10E0D6E0D2EFED70C2EFCD774
:0623720000000000120053
:10237800A4C4F6FFA5C4F7FFA6C4F8FF0900F5CF6B
:1023880000F0005218E0A4C4F6FFA5C4F7FFA6C4E5
:10239800F8FF0900F5CF00F0A2C4E1FFA3C4E2FFF3
:1023A80000C0E6FF0401A24BA32B010EA427000ED8
:1023B800A523A623DDD7A2C4E1FFA3C4E2FFE66AF2
:0223C800120001
:1023CA00A2C4F6FFA3C4F7FFA4C4F8FF0900F5CF1F
:1023DA0000F0005215E0ADB201D0FDD7A2C4F6FF5D
:1023EA00A3C4F7FFA4C4F8FF0900F5CFCAF40EECA2
:1023FA0000F0010E0401A227000EA323A423E0D7B4
:02240A001200BE
:10240C000401A56BA2C4E9FFA3C4EAFFEECFA4F4B8
:10241C00A451000A0FE0A4C4CAF40EEC00F00401AD
:10242C00A52BA551A225E96E000EA321EA6EEECFD5
:06243C00A4F4EED712002B
:102442000D0E0401CA6F0EEC00F00A0E0401CA6FF1
:062452000EEC00F0120088
:10245800020E0C6E350E0D6E0D2EFED70C2EFCD70F
:062468000000000012005C
:10246E00A2C4F6FFA3C4F7FFA4C4F8FF0900F5CF7A
:10247E0000F0005215E0A8B201D0FDD7A2C4F6FFBD
:10248E00A3C4F7FFA4C4F8FF0900F5CFCAF415ECF6
:10249E0000F0010E0401A227000EA323A423E0D70F
:0224AE0012001A
:1024B0000401966B976B010E9A6FF20EA26F010EDC
:1024C000A36F5CDC00C098F401C099F4070E946F10
:1024D000000E956F800E9519006E800E9919005CA4
:1024E00002E19851945DD8B087D15DD1F20E942568
:1024F000E96E010E9521EA6EEECF01F001502C0A33
:102500000CE1520E9625E16E020E9721E26EE66A0C
:10251000966B976B020E9A6F6CD1520E9625E16EF8
:10252000020E9721E26EF20E9425E96E010E9521BE
:10253000EA6EEECF00F000C0E6FF964B972B59D124
:10254000F20E9425E96E010E9521EA6EEECF01F0B0
:1025500001502C0A0CE1BA0E9625E16E020E97216D
:10256000E26EE66A966B976B030E9A6F42D1BA0ED3
:102570009625E16E020E9721E26EF20E9425E96E29
:10258000010E9521EA6EEECF00F000C0E6FF964BFB
:10259000972B2FD1F20E9425E96E010E9521EA6E4C
:1025A000EECF01F001502C0A05E1966B976B040EFB
:1025B0009A6F1FD1F20E9425E96E010E9521EA6EF5
:1025C000EECF00F000C085F3964B972B12D1F20EA0
:1025D0009425E96E010E9521EA6EEECF01F00150CF
:1025E0002C0A0CE1070E9625E16E030E9721E26E90
:1025F000E66A966B976B050E9A6FFBD0070E9625D1
:10260000E16E030E9721E26EF20E9425E96E010E43
:102610009521EA6EEECF00F000C0E6FF964B972BB7
:10262000E8D0F20E9425E96E010E9521EA6EEECF08
:1026300001F001502C0A05E1966B976B060E9A6F1C
:10264000D8D0F20E9425E96E010E9521EA6EEECFF8
:1026500000F000C0CAF2964B972BCBD0F20E942517
:10266000E96E010E9521EA6EEECF01F001502C0AC1
:1026700005E1966B976B070E9A6FBBD0F20E94250F
:10268000E96E010E9521EA6EEECF00F000C088F3EE
:10269000964B972BAED0F20E9425E96E010E952144
:1026A000EA6EEECF01F001502C0A0CE1DF0E962508
:1026B000E16E020E9721E26EE66A966B976B080E4A
:1026C0009A6F97D0DF0E9625E16E020E9721E26E8B
:1026D000F20E9425E96E010E9521EA6EEECF00F020
:1026E00000C0E6FF964B972B84D0F20E9425E96E3E
:1026F000010E9521EA6EEECF01F001502C0A0CE19B
:102700008C0E9625E16E040E9721E26EE66A966BBA
:10271000976B090E9A6F6DD08C0E9625E16E040EA4
:102720009721E26EF20E9425E96E010E9521EA6E74
:10273000EECF00F000C0E6FF964B972B5AD0F20E7A
:102740009425E96E010E9521EA6EEECF01F001505D
:102750002C0A0CE1CF0E9625E16E020E9721E26E57
:10276000E66A966B976B0A0E9A6F43D0CF0E96254A
:10277000E16E020E9721E26EF20E9425E96E010ED3
:102780009521EA6EEECF00F000C0E6FF964B972B46
:1027900030D098C494F499C495F42BD098C494F490
:1027A00099C495F426D09A51010AD8B49FD69A516B
:1027B000020AD8B4C5D69A51030AD8B4EBD69A51B6
:1027C000040AD8B404D79A51050AD8B42AD79A5122
:1027D000060AD8B443D79A51070AD8B45CD79A519D
:1027E000080A83E09A51090AAAE09A510A0AD1E03C
:0E27F000D5D7944B952B6ED69AC400F01200EC
:1027FE000301866B876B000E875D02E1FF0E865D1F
:10280E0012E2890E8625E16E030E8721E26EE66ADC
:10281E00010E8625006E000E8721016E00C086F324
:10282E0001C087F3E8D704018A6B8B6B0301866BBB
:10283E00876B9EAA02D0AFCF89F40401896B010188
:08284E00F06BF16B9D8A120092
:1028560000016051010A08E1480E0401A26F630EEF
:10286600A36F000EA46FAEDD070E0401A26F030E68
:10287600A36F71EC0FF000C01BF301C01CF302C084
:102886001DF303C01EF3000E046E000E056E480E07
:10289600066E850E076E16EC0CF000C017F301C02D
:1028A60018F302C019F303C01AF300C0A2F401C062
:1028B600A3F402C0A4F403C0A5F4B3EC0FF000C067
:1028C60094F401C095F402C096F403C097F494C43E
:1028D60017F395C418F396C419F397C41AF3000EA8
:1028E600046E000E056E480E066E850E076E1BC33F
:1028F60000F01CC301F01DC302F01EC303F016EC6A
:102906000CF094C404F095C405F096C406F097C480
:1029160007F081EC07F000C081F301C082F302C02A
:1029260083F303C084F3000E046E000E056E480E9A
:10293600066E850E076E55EC05F0000E046E000E51
:10294600056E700E066E840E076E16EC0CF094C4BF
:1029560004F095C405F096C406F097C407F09BEC06
:1029660002F000C01BF301C01CF302C01DF303C03C
:102976001EF303018551530A1AE11BC300F01CC361
:1029860001F01DC302F01EC303F0000E046E000E1C
:10299600056E800E066E7F0E076E55EC05F000C0C4
:1029A6001BF301C01CF302C01DF303C01EF31BC3BF
:1029B600A2F41CC3A3F41DC3A4F41EC3A5F41F0EE6
:1029C6000401A66F030EA76F060EA86FD4EC0CF0D9
:1029D600070EA26F030EA36F1F0EA46F030EA56F43
:1029E60078DC03017F6B806B000E805D02E11F0EB9
:1029F6007F5D0BE2E70E7F25E16E020E8021E26E1F
:102A0600200EE66E7F4B802BEFD70201E76BE70EB9
:102A16000401A26F020EA36F1F0EA46F030EA56F13
:102A260058DCE70EA26F020EA36F5C0EA46F000EB9
:102A3600A56FE8EC10F000016051010A16E11F0EC7
:102A46000401A26F030EA36FDEDC200ECA6F0EEC2C
:102A560000F085C3CAF40EEC00F0FD0E0401A26F6F
:102A6600620EA36F000EA46FADDCBA0E0401A26F56
:102A7600020EA36F71EC0FF000C0CBF201C0CCF2D6
:102A860002C0CDF203C0CEF2000E046E000E056E3B
:102A9600480E066E850E076E16EC0CF000C017F396
:102AA60001C018F302C019F303C01AF300C0A2F460
:102AB60001C0A3F402C0A4F403C0A5F4B3EC0FF064
:102AC60000C094F401C095F402C096F403C097F4D4
:102AD60094C417F395C418F396C419F397C41AF35C
:102AE600000E046E000E056E480E066E850E076E0D
:102AF600CBC200F0CCC201F0CDC202F0CEC203F0D0
:102B060016EC0CF094C404F095C405F096C406F0D7
:102B160097C407F081EC07F000C081F301C082F38F
:102B260002C083F303C084F3000E046E000E056E2C
:102B3600480E066E850E076E55EC05F0000E046E07
:102B4600000E056E700E066E840E076E16EC0CF007
:102B560094C404F095C405F096C406F097C407F033
:102B66009BEC02F000C0CBF201C0CCF202C0CDF269
:102B760003C0CEF20201CA51570A1AE1CBC200F0D5
:102B8600CCC201F0CDC202F0CEC203F0000E046E3C
:102B9600000E056E800E066E7F0E076E55EC05F074
:102BA60000C0CBF201C0CCF202C0CDF203C0CEF21F
:102BB600CBC2A2F4CCC2A3F4CDC2A4F4CEC2A5F477
:102BC6001F0E0401A66F030EA76F060EA86FD4ECA6
:102BD6000CF0BA0EA26F020EA36F1F0EA46F030EA7
:102BE600A56F6CEC11F0E70EA26F020EA36F1F0E1D
:102BF600A46F030EA56FE8EC10F0E70EA26F020EAD
:102C0600A36F5E0EA46F000EA56FE8EC10F0000136
:102C16006051010A18E11F0E0401A26F030EA36F93
:102C260006EC12F0200ECA6F0EEC00F0CAC2CAF40F
:102C36000EEC00F0A70E0401A26F620EA36F000E49
:102C4600A46FE5EC11F0CF0E0401A26F020EA36F84
:102C560071EC0FF000C0E3F201C0E4F202C0E5F24D
:102C660003C0E6F200C0A2F401C0A3F402C0A4F4BB
:102C760003C0A5F41F0EA66F030EA76F010EA86F63
:102C8600D4EC0CF0CF0EA26F020EA36F1F0EA46F32
:102C9600030EA56F6CEC11F0E70EA26F020EA36F88
:102CA6001F0EA46F030EA56FE8EC10F00001605133
:102CB600010A07E11F0E0401A26F030EA36F06ECC3
:102CC60012F0200E0201FF6F0301006B066B00017C
:102CD6006051010A2DE1D50E0401A26F620EA36FA9
:102CE600000EA46FE5EC11F0DF0E0401A26F020ED8
:102CF600A36F06EC12F0B30EA26F620EA36F000E66
:102D0600A46FE5EC11F08C0E0401A26F040EA36F04
:102D160006EC12F0E00EA26F620EA36F000EA46F17
:102D2600E5EC11F088C3CAF40EEC00F021EC12F0C9
:102D360000016051010A12E1580E0401A26F630EF0
:102D4600A36F000EA46F37EC12F0E70E0401A26F1A
:0E2D5600020EA36F46EC11F034EC11F01200E7
:102D640096C401F0010E006E015004E0003600909C
:102D7400FF0FFBD700C098F4001E94C4E9FF95C46C
:102D8400EAFF0050EF16120EE9260050EF16B1ECE0
:102D940011F004019851EF12120EE95E2CEC12F0BE
:102DA4009851EF14976F9751000A000ED8A4010EA2
:0C2DB400976FB1EC11F097C400F0120012
:102DC0000401A26BA36B18EC11F00401956B080EC3
:102DD000955D28E29551B00FB96F2AEC06F0C70E49
:102DE0000D6E0D2EFED7000000000401B96B2AEC19
:102DF00006F0100E0401B96F2AEC06F00401966B80
:102E0000800E965D0DE294C4B9F4E8EC05F0C70EAF
:102E10000D6E0D2EFED7000000000401962BF0D79A
:062E2000952BD5D712002E
:102E2600070E0B6E170E0C6E6A0E0D6E0D2EFED76C
:0C2E36000C2EFCD70B2EFAD70000120067
:102E42000401946BEFEC01F0160E0401A26F010E67
:102E5200A36F0C0EA46F61EC11F00050FF0A02E1A7
:102E62000401942B0401170EA26FA36B060EA46F2C
:102E720061EC11F00050FF0A02E10401942B0401FD
:102E8200120EA26F010EA36F070EA46F61EC11F078
:102E92000050FF0A02E10401942B0401110EA26FFB
:102EA200A36B060EA46F61EC11F00050FF0A02E161
:102EB2000401942BE8EC01F09C0E0C6ED70E0D6E03
:0E2EC2000D2EFED70C2EFCD794C400F012008B
:102ED0000900F5CFE6FF0006FBE10106F9E112006B
:102EE000FF0E0F01486F948E949C93988A88846A91
:102EF0008D6A969C070ED26E41919586958492902C
:062F00009292928412007F
:102F06002A0E02018C6F000E8D6FCA0E8E6F040E94
:102F16008F6FFF0E786FFF0E796F000E7A6F000EBF
:102F26007B6FFF0E7C6FFF0E7D6F000E7E6F000EB7
:102F36007F6FFF0E806FFF0E816F000E826F000E97
:102F4600836FA88A900E9C6EA4AA03D0AACF00F025
:042F5600FBD7120093
:102F5A0034EC11F02D0E0401A26F5A0EA36F000E6D
:102F6A00A46F37EC12F0560E0401A26F5B0EA36F2A
:102F7A00000EA46F37EC12F0D40E0401A26F590EA2
:102F8A00A36F000EA46F37EC12F07D0E0401A26F3E
:102F9A005A0EA36F000EA46F37EC12F06A0E0401EA
:102FAA00A26F590EA36F000EA46F37EC12F0150E24
:102FBA000401A26F610EA36F000EA46F37EC12F02A
:102FCA00D20E0401A26F5F0EA36F000EA46F37EC3E
:102FDA0012F01E0E0401A26F5C0EA36F000EA46F06
:102FEA0037EC12F0100E0401A26F5B0EA36F000EF5
:102FFA00A46F37EC12F08F0E0401A26F5E0EA36F5E
:10300A00000EA46F37EC12F0DE0E0401A26F5B0E05
:10301A00A36F000EA46F37EC12F0BB0E0401A26F6F
:10302A005E0EA36F000EA46F37EC12F00C0E0401B3
:10303A00A26F600EA36F000EA46F37EC12F0EF0EB2
:10304A000401A26F5F0EA36F000EA46F37EC12F09B
:10305A00950E0401A26F5F0EA36F000EA46F37ECEA
:08306A0012F034EC11F0120029
:1030720094C4E9FF95C4EAFFEECF96F4000E040172
:10308200976F000E976F000E971902E1200E9619A6
:1030920007E0000E971902E1090E961901E003D02C
:1030A200944B952BE5D7986B996B9A6B9B6B000EA3
:1030B200971902E12D0E961905E19A4B9B2B944B21
:1030C200952B08D0000E971902E12B0E961902E1FA
:1030D200944B952B94C4E9FF95C4EAFFEECF96F486
:1030E200000E976F000E976F96C4C4F494EC01F033
:1030F200005219E098C400F099C401F00A0E046E5F
:10310200000E056EEEEC0BF0300E965D026E000EB8
:103112009759036E02500024986F03500120996F53
:10312200944B952BD7D79A519B1108E098510008E0
:10313200006E99C401F0000E015604D098C400F04C
:0631420099C401F0120027
:103148001C0E02018C6F000E8D6FCA0E8E6F040E5E
:103158008F6FB60E786F1D0E796F000E7A6F000EA6
:103168007B6FD80E7C6F1E0E7D6F000E7E6F000E7B
:103178007F6FFF0E806FFF0E816F000E826F000E53
:10318800836FAD8A900EAC6E948E949C9EAA03D0E9
:08319800AFCF00F0FBD71200DD
:1031A000040E0C6EE40E0D6E0D2EFED70C2EFCD709
:0431B0000000120009
:1031B400210E0401B96F2AEC06F00401B96B2AEC64
:1031C40006F07F0E0401B96F2AEC06F0220E04010A
:1031D400B96F2AEC06F00401B96B2AEC06F0070E6D
:1031E4000401B96F2AEC06F0D30E0401B96F2AEC7E
:1031F40006F0400E0401B96F2AEC06F00401A26B3C
:10320400A36B18EC11F00401946B080E945D28E292
:103214009451B00FB96F2AEC06F0010E0401B96F96
:103224002AEC06F0100E0401B96F2AEC06F0270E02
:103234000D6E0D2EFED7000000000401956B800E6C
:10324400955D0CE2B96BE8EC05F04F0E0D6E0D2E9A
:10325400FED7000000000401952BF1D7942BD5D79D
:103264002E0EB96F2AEC06F00401A26BA36B18ECC6
:0432740011F0120043
:10327800AE0E0401B96F2AEC06F00D0E0B6E2D0E82
:103288000C6ED70E0D6E0D2EFED70C2EFCD70B2E06
:10329800FAD700000000AF0E0401B96F2AEC06F05F
:1032A800070E0B6E170E0C6E6A0E0D6E0D2EFED7E6
:1032B8000C2EFCD70B2EFAD70000B00E0401B96F04
:1032C8002AEC06F00401B96B2AEC06F0070E04019B
:1032D800B96F2AEC06F0200E0401B96F2AEC06F04B
:1032E800020E0401B96F2AEC06F0210E0401B96F31
:1032F8002AEC06F00401B96B2AEC06F07F0E0401F3
:10330800B96F2AEC06F0220E0401B96F2AEC06F018
:103318000401B96B2AEC06F0070E0401B96F2AEC18
:1033280006F0A10E0401B96F2AEC06F0A40E040100
:10333800B96F2AEC06F0A60E0401B96F2AEC06F064
:10334800C80E0401B96F2AEC06F0D30E0401B96F58
:103358002AEC06F0400E0401B96F2AEC06F0D50EEF
:103368000401B96F2AEC06F0800E0401B96F2AEC4B
:1033780006F0A80E0401B96F2AEC06F03F0E04010E
:10338800B96F2AEC06F0D60E0401B96F2AEC06F0E4
:10339800800E0401B96F2AEC06F0D90E0401B96F4A
:1033A8002AEC06F01F0E0401B96F2AEC06F0DA0EBB
:1033B8000401B96F2AEC06F00401B96B2AEC06F097
:1033C800EE0E0401B96F2AEC06F0810E0401B96F04
:1033D8002AEC06F07F0E0401B96F2AEC06F02E0ED7
:1033E8000401B96F2AEC06F0DB0E0401B96F2AEC70
:1033F80006F0400E0401B96F2AEC06F08D0E0401A8
:10340800B96F2AEC06F0140E0401B96F2AEC06F025
:0C341800AF0E0401B96F2AEC06F01200A0
:103424008D0E0401B96F2AEC06F0140E0401B96F75
:103434002AEC06F0AF0E0401B96F2AEC06F0120074
:103444003D0E0B6EE10E0C6E3F0E0D6E0D2EFED773
:0E3454000C2EFCD70B2EFAD700000000120041
:1034620004019D6B9E6B9F6BA06BA16B94C4A0F437
:1034720095C4A1F494C4A2F495C4A3F418EC11F079
:1034820038D104019F519625E96E000E9721EA6E0C
:10349200EE50000A46E0050EA15D43E29F519625DB
:1034A200E96E000E9721EA6E200EEE5C9D6FA05130
:1034B200780809E294C4A0F4A12B94C4A2F4A1C494
:1034C200A3F418EC11F004019E6B060E9E5D25E23A
:1034D200060E006E000E016E026E036E9DC404F0B5
:1034E200000E056E066E076E4AEC01F0420E0026D3
:1034F200570E0122000E02229E510024F66E000E8B
:103502000120F76E000E0220F86E0900F5CFB9F423
:10351200E8EC05F004019E2BD8D7060EA0279F2BBE
:10352200B0D7F4D096C4A2F497C4A3F4BEEC0EF0C4
:1035320000C099F401C09AF49F6B9F519625E96EE1
:10354200000E9721EA6EEE50000AD8B475D00F0E25
:103552009F5D72E29F519625E96E000E9721EA6EF9
:10356200200EEE5C9D6FA0C4A2F4A1C4A3F418ECDB
:1035720011F004019E6B080E9E5D25E2040E026EA0
:103582009DC400F0000E016E025005E0003600906E
:103592000136FF0FFAD79E510026000E0122520E6D
:1035A2000024F66E510E0120F76E000EF86E000E2A
:1035B20001BEFF0EF8220900F5CFB9F4E8EC05F0E0
:1035C20004019E2BD8D7A0C4A2F4A151010FA36F6E
:1035D20018EC11F004019E6B080E9E5D29E2040EA8
:1035E200026E9DC400F0000E016E025005E000362E
:1035F20000900136FF0FFAD79E510026000E0122DD
:10360200080E0026000E0122520E0024F66E510E04
:103612000120F76E000EF86E000E01BEFF0EF822BA
:103622000900F5CFB9F4E8EC05F004019E2BD4D7DC
:10363200080EA0279F2B81D769D096C4A2F497C405
:10364200A3F4BEEC0EF000C09BF401C09CF4800E0B
:10365200026E800E0118025C02E10050000847E28F
:103662009E6B800E006E800E9C19005C02E19B51E5
:103672009E5D3DE2070E9E25996F9A6B000E9A237E
:103682009B51995F9C519A5B040E006E005005E0BD
:10369200993799919A37FF0FFAD79E519625E96E7D
:1036A200000E9721EA6EEECF01F001C09DF40150A9
:1036B2002F080BE23A0E9D5D08E299C4A2F4300E87
:1036C2009D5DA36F4DEC10F010D09D512E0A07E1C5
:1036D20099C4A2F40A0EA36F4DEC10F006D099C45F
:1036E200A2F4200EA36F4DEC10F09E2BBAD70ED091
:1036F2000DD004019851010AD8B4C3D69851020AD8
:0E370200D8B410D79851030A98E0F2D71200FD
:10371000200E0401B96F2AEC06F00401B96B2AEC03
:1037200006F0210E0401B96F2AEC06F094C4B9F436
:103730002AEC06F004019451070FB96F2AEC06F049
:10374000220E0401B96F2AEC06F095C4B9F42AECF4
:1037500006F004019551010FB96F2AEC06F004013F
:10376000976B986B800E9819006E800E005C02E1DA
:10377000070E975D24E2030E006E000E016E96C4E4
:1037800004F0000E056EEEEC0BF04D0E0024E96E19
:10379000000E0120EA6E9751EE24F66E9851EE204D
:1037A000F76E000E98BFFF0EEE20F86E0900F5CF01
:1037B000B9F4E8EC05F00401974B982BD3D712002D
:1037C000DBEC0EF094C424F095C425F0E4EC0EF08C
:1037D000300E0401A26F5F0EA36F000EA46F37ECD2
:1037E00012F094C4A2F495C4A3F4960E0401A46F3D
:1037F000040EA56FF0EC0EF0960EA26F040EA36FF0
:1038000046EC11F08D0EA26F620EA36F000EA46F36
:1038100037EC12F06CEC0FF00050000A04E10201EA
:0C38200060B301D0F7D7DBEC0EF0120013
:10382C0094C404F095C405F004019851991124E056
:10383C00010E985F000E995B04C002F005C003F006
:10384C00044A052A96C400F097C401F0964B972BB6
:10385C0000C0E9FF01C0EAFF02C0E1FF03C0E2FFC4
:10386C00EECFE6FF02C0E9FF03C0EAFFEECF00F0A7
:10387C00005201E101D0D8D798C400F099C401F0EE
:10388C00010E985F000E995B0050011008E004C017
:10389C00E1FF05C0E2FFE66A044A052AEDD794C4AD
:0838AC0000F095C401F01200C8
:1038B40094C400F00032009E0032009E0032009E4C
:1038C4000032009E320E0024F66E620EF76E000E79
:1038D400F722000EF86E000EF8220900F5CF00F072
:1038E40095C4E1FF96C4E2FF00C0E6FF010E0401A7
:1038F4009525E16E000E9621E26E0F0E9415006E72
:10390400320E0024F66E620EF76E000EF722000EE1
:10391400F86E000EF8220900F5CF00F000C0E6FFB3
:10392400020E9525E16E000E9621E26EE66A120003
:103934000401996B95AF0BD0010E996F2D0E030105
:103944001F6F0401941F951F944B952B04D0996B02
:10395400200E03011F6F94C400F095C401F00132DE
:103964000032019E01320032019E01320032019E7A
:1039740001320032019E00C096F40A0E046E6FEC10
:1039840006F00A0E046E6FEC06F008C000F0300E6C
:103994000024016E01C020F30150300A03E1030149
:1039A400200E206F03010A0E046E96C400F06FEC23
:1039B40006F008C000F0300E0024216F94C497F480
:1039C40095C498F40F0E04019415006E95C401F08B
:1039D400000E011600C097F401C098F4710E046E35
:1039E400020E056EEEEC0BF000C09AF401C09BF4DD
:1039F4009AC497F49BC498F42E0E0301226FE80E28
:103A0400046E030E056E9AC400F09BC401F054ECDE
:103A140006F0300E0024236F640E046E000E056E53
:103A24009AC400F09BC401F054EC06F00A0E046E34
:103A3400000E056E54EC06F008C000F009C001F059
:103A4400300E0024246F256B266B276B200E040197
:103A5400A26F030EA36F7BEC0FF09951010A14E1DE
:103A640096C400F0000E016EE80E046E030E056E9F
:103A7400EEEC0BF097510024206E98510120216E3A
:103A8400000E226E236E18D096C400F0000E016E54
:103A9400E80E046E030E056EEEEC0BF09751002653
:103AA4009851012200500008206E01C021F0000E40
:0E3AB4002156000E226E236E99C400F01200FF
:103AC20096C401F0010E006E015004E00036009031
:103AD200FF0FFBD700C09AF4001E00C099F494C4F3
:103AE200E9FF95C4EAFF0050EF16120EE926040121
:103AF200986B9851070816E398C400F097C401F038
:103B0200005004E00132019EFF0FFBD79951EF16DE
:103B120001A002D09A51EF122CEC12F09A51EF123E
:103B2200982BE7D7120EE95E3FEC11F03FEC11F053
:023B320012007F
:103B340096C401F0010E006E015004E000360090BE
:103B4400FF0FFBD700C09AF4001C0401996F986B17
:103B540094C4E9FF95C4EAFF976B9751070824E3DF
:103B64009951EF16120EE9269951EF16E1EC10F077
:103B74009A51EF12E1EC10F0120EE95E9A51EF1433
:103B8400006E0CE097C401F0010E006E015004E0D9
:103B940000360090FF0FFBD7005098133FEC11F054
:0E3BA4003FEC11F0972BD9D798C400F0120017
:103BB200010E04019E6F220EA26F620EA36F000E11
:103BC200A46F37EC12F094C4A2F4950E0401A36F13
:103BD200040EA46FA5EC10F0950EA26F040EA36F55
:103BE20046EC11F0400EA26F630EA36F000EA46F9D
:103BF20037EC12F0F40E0401A26F620EA36F000EF6
:103C0200A46F37EC12F0A0EC01F094C4C4F4F6EC0B
:103C120001F000C09EF40050000A0CE07F0E040187
:103C2200A26F620EA36F000EA46F37EC12F00401B4
:103C32009E6B0CD00401EA0EA26F620EA36F000EFF
:103C4200A46F37EC12F0010E04019E6F74EC02F0C7
:0A3C520034EC11F09EC400F01200E3
:103C5C000001EE6BEF6B000EEF5D02E1FF0EEE5D0F
:103C6C0012E2F00EEE25E16E000EEF21E26EE66A36
:103C7C00010EEE25006E000EEF21016E00C0EEF07D
:103C8C0001C0EFF0E8D7EE6BEF6B000EEF5D02E1D9
:103C9C00600EEE5D12E2F20EEE25E16E010EEF21EA
:103CAC00E26EE66A010EEE25006E000EEF21016E4B
:103CBC0000C0EEF001C0EFF0E8D7EE6BEF6B000E3A
:103CCC00EF5D02E1600EEE5D12E21F0EEE25E16E7D
:103CDC00030EEF21E26EE66A010EEE25006E000E79
:103CEC00EF21016E00C0EEF001C0EFF0E8D7070E37
:103CFC000401A26F030EA36FA30EA46F630EA56F36
:103D0C00000EA66FBCEC11F0BA0E0401A26F020EED
:103D1C00A36F9F0EA46F630EA56F000EA66FBCEC75
:103D2C0011F0CF0E0401A26F020EA36F9B0EA46FB5
:103D3C00630EA56F000EA66FBCEC11F002015E6B5A
:103D4C005F6B0001EE6BEF6BA4AA02D0AACF61F2FD
:103D5C000201616B626B636BA38A266A276A12008D
:103D6C00000E0401951902E1000E941937E094C479
:103D7C00E9FF95C4EAFFEE5231E096C4A2F497C471
:103D8C00A3F4BEEC0EF000C0A6F494C4A2F495C447
:103D9C00A3F496C4A4F497C4A5F43BEC0FF0000E66
:103DAC00011802E1000E001805E194C400F095C45E
:103DBC0001F016D0010E04019425A26F000E95217E
:103DCC00A36F96C4E9FF97C4EAFFEECFA4F493EC7B
:103DDC0011F000C094F401C095F4C2D7006A016AD6
:023DEC001200C3
:103DEE00620E0201646F020E656F000E666F000EAA
:103DFE00676F400E686F030E696F000E6A6F000EDC
:103E0E006B6FFF0E6C6FFF0E6D6F000E6E6F000E00
:103E1E006F6FFF0E746FFF0E756FFF0E766FFF0ED6
:103E2E00776FEC0E846F030E856FC40E866F040ED3
:103E3E00876FE80E886F040E896F000E8A6F000E72
:103E4E008B6F959295908C928C9095829580739EA7
:083E5E00739C380E726E120015
:103E660000C01BF001C01AF0E1CF1CF0E2CF1DF03C
:103E7600A4AA8BD0A3AA89D0AACF61F29CA202D011
:103E86009C989C889CA404D0AACF61F20201616B25
:103E96000001EF51000802E1EE51FF0819E2EEC001
:103EA6005EF2EFC05FF2AACF61F20201616BF00E23
:103EB6000001EE25E16E000EEF21E26EE66AEE6B82
:103EC600EF6B010E0201626F000E636FA39A5DD065
:103ED60044D002016151520A04E1010E266E000E21
:103EE600276E53D0020161514D0A04E1020E266E7F
:103EF600000E276E4AD002016151430A04E1030E07
:103F0600266E000E276E240E0001F06F470EF16F2D
:103F1600500EF26F520EF36F4D0EF46F430EF56FA7
:103F2600050EEE6F000EEF6F30D00001F00EEE259D
:103F3600E16E000EEF21E26E61C2E6FFEEC05EF2B8
:103F4600EFC05FF2010EEE25006E000EEF21016E4E
:103F560000C0EEF001C0EFF018D0000E271802E105
:103F6600000E2618B6E0000E271802E1010E2618EC
:103F7600B9E0000E271802E1020E2618BCE0000E7A
:103F8600271802E1030E2618D0E09EAA4BD09DAA60
:103F960049D0AFCF89F4ACA203D0AC98AC88AC9230
:103FA600ACA402D0AFCF89F4040189510D0A0AE00E
:103FB600000E006E03018751005C02E186513F0846
:103FC60001E319D0010E0101F06F000EF16F9D9A09
:103FD600890E03018625E16E030E8721E26EE66AED
:103FE60086C38AF487C38BF4866B876BAFCF89F45D
:103FF6000401896B17D0890E03018625E16E030E35
:104006008721E26E89C4E6FF86C38AF487C38BF4F0
:10401600010E8625006E000E8721016E00C086F314
:1040260001C087F31BC000F01AC001F01CC0E1FFFD
:064036001DC0E2FF1100B5
:10403C0000C019F001C018F0156ED8CF16F0E0CF03
:10404C0017F0F2AA1DD0F2A41BD06D0ED76E840E01
:10405C00D66E010E245C006E000E2558016E00C059
:10406C0024F001C025F0800E2518006E800E005C37
:10407C0002E1010E245C03E202016083F29AF294E5
:10408C001750E06E1650D86E153A153819C000F05E
:06409C0018C001F0100045
:1040A200D4EC31F070EC17F0010E0001606F8990D2
:1040B20089926D0E6B6F000E6C6F8980948E949C4A
:1040C200959C958A21EC17F000C0EDF00050040A8F
:1040D20003E10201608D02D00201609D7E86040E22
:1040E2007F6EE10EB06EAD84A4EC18F0070E0B6E7D
:1040F200170E0C6E6A0E0D6E0D2EFED70C2EFCD70F
:104102000B2EFAD700007C86040E7D6EE10EAB6E9C
:10411200A88483EC17F0ADEC17F021EC12F0A70E97
:104122000401A26F600EA36F000EA46FE5EC11F004
:10413200E50E0401A26F5E0EA36F000EA46FE5EC04
:1041420011F0300E0001ED250401CA6F0EEC00F0F3
:104152000001ED51040A0AE1500E0401A26F630E40
:10416200A36F000EA46FE5EC11F009D0CA0E040192
:10417200A26F620EA36F000EA46FE5EC11F021ECAA
:1041820012F0A39A9D9AF28CD08E1F0E0B6E710EB6
:104192000C6E1E0E0D6E0D2EFED70C2EFCD70B2EA6
:1041A200FAD700008982FFEC13F08A980D0E0B6E8D
:1041B2002D0E0C6ED70E0D6E0D2EFED70C2EFCD7CB
:1041C2000B2EFAD700000000F28E610E0401A26FDE
:1041D200620EA36F000EA46F37EC12F0520E0401B0
:1041E200A26F620EA36F000EA46FE5EC11F07B0EBE
:1041F2000401A26F630EA36F000EA46FE5EC11F031
:10420200810E0401A26F630EA36F000EA46F37EC40
:1042120012F00D0E0B6E2D0E0C6ED70E0D6E0D2EB6
:10422200FED70C2EFCD70B2EFAD700000000000E92
:104232000101F11902E1010EF01912E1280E040147
:10424200A26F600EA36F000EA46F37EC12F0890EFE
:104252000401A26F030EA36F46EC11F034EC11F0CF
:10426200FFEC13F0060E0401A26F630EA36F000EA3
:10427200A46FE5EC11F00F0E0401A26F630EA36FA1
:10428200000EA46F37EC12F0310E0B6EB40E0C6EF2
:10429200650E0D6E0D2EFED70C2EFCD70B2EFAD707
:1042A20000000000000E0101F11902E1010EF019F7
:1042B20012E15C0E0401A26F600EA36F000EA46FE8
:1042C20037EC12F0890E0401A26F030EA36F46ECC5
:1042D20011F034EC11F08A881F0E0B6E710E0C6E09
:1042E2001E0E0D6E0D2EFED70C2EFCD70B2EFAD7FE
:1042F200000034EC11F00D0E0401A26F5F0EA36FEB
:10430200000EA46F37EC12F013EC17F00001616B92
:10431200626B800E0401946F0F0E956F020E966F02
:10432200B2EC16F0D0EC18F0800E946F0F0E956F71
:10433200020E966F330E976F61EC1DF0D0EC18F001
:10434200800E946F0F0E956F020E966F9AEC1DF011
:1043520000C089F4D0EC18F0420EA26F620EA36F77
:10436200000EA46F37EC12F003011F6B89C494F4A2
:104372001F0E0401956F030E966F5AEC1CF01F0E70
:10438200A26F030EA36F46EC11F0200EA26F630E14
:10439200A36F000EA46F37EC12F003017F6B806BEA
:1043A200000E805D02E1060E7F5D2AE2800E0401AE
:1043B200946F0F0E956F020E966F9AEC1DF000C06F
:1043C20089F4D0EC18F0630E03017F25E16E000E34
:1043D2008021E26E89C4E6FF1F6B89C494F41F0E2C
:1043E2000401956F030E966F5AEC1CF01F0EA26F1C
:1043F200030EA36F46EC11F003017F4B802BD0D745
:10440200180E0401A26F630EA36F000EA46F37ECA7
:1044120012F0800E0401946F0F0E956F020E966FCC
:104422009AEC1DF000C089F403011F6B89C494F457
:104432001F0E0401956F030E966F5AEC1CF01F0EAF
:10444200A26F030EA36F46EC11F034EC11F0100EC4
:104452000401A26F620EA36F000EA46F37EC12F07C
:10446200800E0401946F0F0E956F020E966FB2ECE0
:1044720016F0800E946F0F0E956F020E966FCC0E93
:10448200976F61EC1DF0800E946F0F0E956F020E08
:10449200966F440E976F61EC1DF0D0EC18F0800E11
:1044A200946F0F0E956F020E966FB2EC16F0800E9F
:1044B200946F0F0E956F020E966FCC0E976F61EC94
:1044C2001DF0800E946F0F0E956F020E966FBE0E4A
:1044D200976F61EC1DF0250E0B6E870E0C6E8B0E26
:1044E2000D6E0D2EFED70C2EFCD70B2EFAD7000028
:1044F2000000800E946F0F0E956F020E966F9AEC6D
:104502001DF000C01EF0000E1F6E800E946F0F0E85
:10451200956F020E966F9AEC1DF000C003F0026ACE
:104522001E500224006E1F500320016E00C059F07D
:1045320001C05AF000C094F401C095F49AEC1CF04A
:104542001F0EA26F030EA36F7BEC0FF01F0EA26F64
:10455200030EA36FBEEC0EF000C093F201C094F202
:104562001F0E0024A26F030E0120A36F910EA46FF1
:10457200630EA56F000EA66FBCEC11F01F0E0401B6
:10458200A26F030EA36F46EC11F034EC11F034EC81
:1045920011F0E90E0401A26F600EA36F000EA46F6A
:1045A20037EC12F0780E746E21DC31EC01F0005021
:1045B200000A01E1FAD7070E0B6E170E0C6E6A0E97
:1045C2000D6E0D2EFED70C2EFCD70B2EFAD7000047
:1045D200780E0201956F780E0401946FD9EC1DF0EC
:1045E20000C093F2000E0201946F740E03017F6FFC
:1045F200000E806F000E805D02E1820E7F5D25E27B
:104602007FC394F4D9EC1DF000C093F2000E0201B6
:10461200946F070E0B6E170E0C6E6A0E0D6E0D2E3A
:10462200FED70C2EFCD70B2EFAD70000000E006E20
:104632009451005C02E19351000801E206D0020E9F
:1046420003017F27000E8023D5D7070E0B6E170EAE
:104652000C6E6A0E0D6E0D2EFED70C2EFCD70B2E95
:10466200FAD70000000E0201941902E1000E93191C
:104672000DE18F0E0401A26F600EA36F000EA46FF6
:1046820037EC12F089828990A8EF28F0700E0401AD
:10469200A26F620EA36F000EA46FE5EC11F09A0EEA
:1046A2000401A26F620EA36F000EA46F37EC12F02A
:1046B2003CEC19F0070E0B6E170E0C6E6A0E0D6EA7
:1046C2000D2EFED70C2EFCD70B2EFAD70000BF0EF4
:1046D2000401A26F620EA36F000EA46F37EC12F0FA
:1046E20012EC1AF0070E0B6E170E0C6E6A0E0D6EA0
:1046F2000D2EFED70C2EFCD70B2EFAD70000FE0E85
:104702000201906FFF0E916F6D0E00016B6F000E34
:104712006C6F83A601D0CBD1F28EDAEC18F06BC0AD
:10472200A2F46CC0A3F42B0E0401A46F610EA56F5A
:10473200000EA66FBCEC11F00401946B956B6BC07C
:1047420096F46CC097F4010E986F31EC1AF06BC0BE
:10475200A2F46CC0A3F446EC11F034EC11F022EC9C
:104762001AF022EC1AF022EC1AF06BC0A2F46CC020
:10477200A3F4810E0401A46F610EA56F000EA66F53
:10478200BCEC11F06BC0A2F46CC0A3F446EC11F0C7
:1047920034EC11F0010E0401946F010E956F6BC0A1
:1047A20096F46CC097F4010E986F31EC1AF0140E67
:1047B200946F000E956FE0EC1BF0DAEC18F06BC012
:1047C200A2F46CC0A3F4410E0401A46F610EA56FA4
:1047D200000EA66FBCEC11F06BC0A2F46CC0A3F487
:1047E20046EC11F034EC11F00401946B956B6BC044
:1047F20096F46CC097F4010E986F31EC1AF06BC00E
:10480200A2F46CC0A3F4C80EA46F5A0EA56F000EDA
:10481200A66FBCEC11F0010E0401946F010E956FAE
:104822006BC096F46CC097F4010E986F31EC1AF0DD
:10483200140E946F000E956FE0EC1BF0DAEC18F09A
:104842006BC0A2F46CC0A3F4EA0E0401A46F610E63
:10485200A56F000EA66FBCEC11F06BC0A2F46CC089
:10486200A3F446EC11F034EC11F00401946B956B57
:104872006BC096F46CC097F4010E986F31EC1AF08D
:104882006BC0A2F46CC0A3F46C0EA46F610EA56F92
:10489200000EA66FBCEC11F0010E0401946F030E22
:1048A200956F6BC096F46CC097F4010E986F31EC63
:1048B2001AF0140E946F000E956FE0EC1BF0DAEC18
:1048C20018F06BC0A2F46CC0A3F4D50E0401A46F5F
:1048D200610EA56F000EA66FBCEC11F06BC0A2F4C6
:1048E2006CC0A3F446EC11F034EC11F00401946BAB
:1048F200956B6BC096F46CC097F4010E986F31EC17
:104902001AF06BC0A2F46CC0A3F4AB0EA46F610EDC
:10491200A56F000EA66FBCEC11F0010E0401946F9E
:10492200010E956F6BC096F46CC097F4020E986FEF
:1049320031EC1AF0140E946F000E956FE0EC1BF040
:10494200DAEC18F0040E0B6E0C0E0C6E330E0D6EBC
:104952000D2EFED70C2EFCD70B2EFAD7000000002E
:104962006BC0A2F46CC0A3F4960E0401A46F610E96
:10497200A56F000EA66FBCEC11F06BC0A2F46CC068
:10498200A3F446EC11F0946B956B6BC096F46CC07B
:1049920097F4010E986F31EC1AF06BC0A2F46CC060
:1049A200A3F4660EA46F630EA56F000EA66FBCEC97
:1049B20011F06BC0A2F46CC0A3F446EC11F034EC1D
:1049C20011F0010E0401946F010E956F6BC096F405
:1049D2006CC097F4030E986F31EC1AF0140E946FBA
:1049E200000E956FE0EC1BF0DAEC18F0040E0B6E83
:1049F2000C0E0C6E330E0D6E0D2EFED70C2EFCD748
:104A02000B2EFAD7000000006BC0A2F46CC0A3F416
:104A1200760E0401A46F600EA56F000EA66FBCECAB
:104A220011F06BC0A2F46CC0A3F446EC11F0080EB6
:104A3200946F010E956F030E966F88EC1BF0100EAB
:104A4200946F010E956F010E966F88EC1BF0200E8D
:104A5200946F010E956F020E966F88EC1BF0140E88
:104A6200946F000E956FE0EC1BF0DAEC18F06BC05F
:104A7200A2F46CC0A3F4C00E0401A46F610EA56F72
:104A8200000EA66FBCEC11F06BC0A2F46CC0A3F4D4
:104A920046EC11F034EC11F0FF0E0401946FE0ECDF
:104AA20016F0140E946F000E956FE0EC1BF0DAEC2A
:104AB20018F0F28CF28CF28E898089928970800EC5
:104AC2000401946F0F0E956F020E966FB2EC16F002
:104AD200800E946F0F0E956F020E966FCC0E976F2D
:104AE20061EC1DF0800E946F0F0E956F020E966FA3
:104AF200440E976F61EC1DF0D0EC18F0800E946FAD
:104B02000F0E956F020E966FB2EC16F0800E946F38
:104B12000F0E956F020E966FCC0E976F61EC1DF023
:104B2200800E946F0F0E956F020E966FBE0E976FEA
:104B320061EC1DF0130E0B6E440E0C6E440E0D6EE6
:104B42000D2EFED70C2EFCD70B2EFAD70000800EAE
:104B5200946F0F0E956F020E966F9AEC1DF000C0C7
:104B62001EF0000E1F6E800E946F0F0E956F020ED8
:104B7200966F9AEC1DF000C003F0026A1E500224E8
:104B8200006E1F500320016E00C059F001C05AF0A0
:104B920000C094F401C095F49AEC1CF000C092F2AB
:104BA2001F0EA26F030EA36F7BEC0FF01F0EA26FFE
:104BB200030EA36FBEEC0EF000C093F201C094F29C
:104BC200020E005C026E000E0158036E1F0E0224DC
:104BD200E96E030E0320EA6E300EEE5C036E03C034
:104BE20004F004360490043604900436049004362B
:104BF2000490010E005C026E000E0158036E1F0E3F
:104C02000224E96E030E0320EA6E300EEE5C026EA1
:104C1200025004240201966F050E005C026E000E23
:104C22000158036E1F0E0224E96E030E0320EA6E82
:104C3200300EEE5C046E04C002F0023602900236C0
:104C420002900236029002360290040E005E000EBE
:104C5200015A1F0E0024E96E030E0120EA6E300E87
:104C6200EE5C006E005002249B6F9C0E0401A26F4A
:104C7200020EA36FFE0EA46F610EA56F000EA66F4B
:104C8200BCEC11F0A50E0401946F020E956F1F0E7D
:104C9200966F030E976F010E0201935D0401986FE8
:104CA200000E020194590401996F16EC1CF09C0E3F
:104CB200A26F020EA36F46EC11F0270E0201AB6F3A
:104CC200090E0401CA6F15EC00F0070E0401A26F71
:104CD200030EA36F870EA46F630EA56F000EA66F5F
:104CE200BCEC11F0BA0E0401A26F020EA36F8C0E7F
:104CF200A46F630EA56F000EA66FBCEC11F0CF0E71
:104D02000401A26F020EA36F960EA46F630EA56F2D
:104D1200000EA66FBCEC11F02EEC1EF0B50E0401D5
:104D2200A26F5F0EA36F000EA46F37EC12F08972B0
:104D3200430E0B6EF70E0C6EAD0E0D6E0D2EFED7E2
:104D42000C2EFCD70B2EFAD7000E0201631902E1DA
:104D5200010E6219D8A485D00101A16BF29A83B623
:104D620014D083B412D0740E0401A26F5F0EA36F2D
:104D7200000EA46F37EC12F0F00E0401A26F000EC9
:104D8200A36F46EC11F034EC11F01F0E0401A26F78
:104D9200030EA36F5F0EA46F630EA56F000EA66FC6
:104DA200BCEC11F0F00E0401946F000E956F1F0E13
:104DB200966F030E976FB6EC1EF000C097F201C01B
:104DC20098F2000E026E0150025C02E100500008EF
:104DD20047E203017F6B806B000E805D02E15F0E94
:104DE2007F5D15E2F20E7F25E16E010E8021E26EFB
:104DF2007F5102019725E96E03018051020198213A
:104E0200EA6EEECFE6FF03017F4B802BE5D75F0E04
:104E120002019725E16E000E9821E26EE66A58ECD7
:104E220012F000C05BF000500A0A1AE12BEC14F0F9
:104E3200DF0E0401946F020E956F39EC18F000C07A
:104E420099F201C09AF200016051000A09E1300EA4
:104E52000401A26F630EA36F000EA46F37EC12F071
:104E620012D0530E0401A26F5F0EA36F000EA46F47
:104E720037EC12F0420E0401A26F600EA36F000E17
:104E8200A46FE5EC11F06D0E00016B6F000E6C6FFC
:104E9200010E02019015016E91C202F0000E02167F
:104EA200000E021802E1000E011829E16BC0A2F403
:104EB2006CC0A3F4570E0401A46F610EA56F000E1F
:104EC200A66FBCEC11F090C2A2F491C2A3F40C0E36
:104ED20000016B250401A46F000E00016C21040186
:104EE200A56FF0EC0EF0010E946F956B6BC096F40B
:104EF2006CC097F4010E986F31EC1AF00CD00401DB
:104F0200010E946F956B9C0E966F020E976F010EB9
:104F1200986F31EC1AF06D0E00016B6F000E6C6F22
:104F22006BC0A2F46CC0A3F4FF0E0401A46F600E68
:104F3200A56F000EA66FBCEC11F0070E00016B25E9
:104F42000401A26F000E00016C210401A36F070E81
:104F5200A46F030EA56F6CEC11F06BC0A2F46CC0D1
:104F6200A3F4BEEC0EF000C093F201C094F2000E66
:104F7200015C02E1140E005C0CE20201935100019B
:104F82006B25E16E0201945100016C21E26E200E4C
:104F9200E66E010E0401946F010E956F6BC096F4DC
:104FA2006CC097F4010E986F31EC1AF06D0E00018F
:104FB2006B6F000E6C6F6BC0A2F46CC0A3F4BD0EDD
:104FC2000401A46F600EA56F000EA66FBCEC11F079
:104FD200070E00016B250401A26F000E00016C2177
:104FE2000401A36FBA0EA46F020EA56F6CEC11F050
:104FF2006BC0A2F46CC0A3F4BEEC0EF000C093F23E
:1050020001C094F2000E015C02E1140E005C0CE29D
:105012000201935100016B25E16E020194510001DE
:105022006C21E26E200EE66E010E0401946F020EF8
:10503200956F6BC096F46CC097F4010E986F31ECCB
:105042001AF06D0E00016B6F000E6C6F6BC0A2F454
:105052006CC0A3F4D30E0401A46F600EA56F000E02
:10506200A66FBCEC11F0070E00016B250401A26FC4
:10507200000E00016C210401A36FCF0EA46F020E7B
:10508200A56F6CEC11F06BC0A2F46CC0A3F4BEEC83
:105092000EF000C093F201C094F2000E015C02E136
:1050A200140E005C0CE20201935100016B25E16ECB
:1050B2000201945100016C21E26E200EE66E010E97
:1050C2000401946F030E956F6BC096F46CC097F455
:1050D200010E986F31EC1AF00201904B912B83B6BE
:1050E20005D083A403D0010E0001606F83B404D005
:1050F20083A602D00001606BFFEC13F03D0E0B6E35
:10510200E10E0C6E3F0E0D6E0D2EFED70C2EFCD74F
:105112000B2EFAD700000000000EF11902E1010E79
:10512200F01914E1620E0401A26F5E0EA36F000E6D
:10513200A46F37EC12F00301C96B890E0401A26F50
:10514200030EA36F46EC11F034EC11F0B7D4FFD785
:1063A80010EE1EF0430E006E010E016E9B0EF66E8F
:0E63B8005B0EF76E000EF86E68EC17F0120028
:10515200000000000000000000000000000000004D
:10516200000000F8000000000000003330000000E2
:1051720000100C06100C06000000000000000000E9
:1051820040C07840C0784000043F04043F0404005B
:10519200007088FC08300000001820FF211E00006B
:1051A200F008F000E018000000211C031E211E0080
:1051B20000F00888700000001E2123241927211006
:1051C20010160E00000000000000000000000000A9
:1051D200000000E018040200000000071820400050
:1051E20000020418E0000000004020180700000040
:1051F200404080F0804040000202010F01020200A4
:10520200000000F0000000000101011F0101010087
:10521200000000000000000080B0700000000000EC
:105222000000000000000000000101010101010175
:10523200000000000000000000303000000000000C
:1052420000000000806018040060180601000000E1
:1052520000E010080810E000000F102020100F00DE
:10526200001010F8000000000020203F2020000065
:1052720000700808088870000030282422213000BD
:1052820000300888884830000018202020110E00C5
:105292000000C02010F8000000070424243F24006E
:1052A20000F80888880808000019212020110E0043
:1052B20000E0108888180000000F112020110E0055
:1052C20000380808C83808000000003F000000004D
:1052D2000070880808887000001C222121221C000E
:1052E20000E010080810E0000000312222110F0037
:1052F200000000C0C00000000000003030000000CC
:10530200000000800000000000008060000000003B
:105312000000804020100800000102040810200054
:10532200404040404040400004040404040404009F
:105332000008102040800000002010080402010034
:10534200007048080808F000000000303601000034
:10535200C030C828E810E0000718272423140B00E7
:105362000000C038E0000000203C23020227382061
:1053720008F8888888700000203F202020110E0045
:10538200C03008080808380007182020201008003C
:1053920008F808080810E000203F202020100F0025
:1053A20008F88888E8081000203F202023201800F1
:1053B20008F88888E8081000203F20000300000059
:1053C200C03008080838000007182020221E0200FA
:1053D20008F808000008F808203F210101213F20B9
:1053E200000808F8080800000020203F20200000E4
:1053F20000000808F8080800C08080807F000000D4
:1054020008F888C028180800203F2001263820000C
:1054120008F8080000000000203F20202020300073
:1054220008F8F800F8F80800203F003F003F20008D
:1054320008F830C00008F808203F200007183F0095
:10544200E01008080810E0000F10202020100F00C4
:1054520008F808080808F000203F210101010000B7
:10546200E01008080810E0000F18242438504F00FC
:1054720008F8888888887000203F2000030C3020BC
:1054820000708808080838000038202121221C00FA
:10549200180808F8080818000000203F2000000043
:1054A20008F808000008F808001F202020201F002C
:1054B2000878880000C83808000007380E0100008C
:1054C200F80800F80008F800033C0700073C030056
:1054D200081868808068180820302C03032C3020BC
:1054E2000838C800C83808000000203F200000002B
:1054F20010080808C8380800203826212020180083
:10550200000000FE020202000000007F4040400056
:10551200000C30C000000000000000010638C0008E
:1055220000020202FE000000004040407F00000036
:10553200000004020202040000000000000000005B
:105542000000000000000000808080808080808059
:105552000002020400000000000000000000000041
:1055620000008080808000000019242222223F2037
:1055720008F8008080000000003F112020110E007A
:105582000000008080800000000E11202020110009
:10559200000000808088F800000E112020103F20BB
:1055A2000000808080800000001F2222222213003F
:1055B200008080F0888888180020203F202000008A
:1055C2000000808080808000006B9494949360003F
:1055D20008F8008080800000203F210000203F204A
:1055E20000809898000000000020203F202000004A
:1055F200000000809898000000C08080807F00003A
:1056020008F8000080808000203F24022D30200016
:10561200000808F8000000000020203F20200000C1
:105622008080808080808000203F20003F20003FDB
:105632008080008080800000203F210000203F20E9
:105642000000808080800000001F202020201F009A
:10565200808000808000000080FFA12020110E00C9
:105662000000008080808000000E112020A0FF80BA
:10567200808080008080800020203F212000010067
:1056820000008080808080000033242424241900BC
:10569200008080E0808000000000001F20200000C9
:1056A2008080000000808000001F202020103F200A
:1056B200808080000080808000010E30080601009A
:1056C20080800080008080800F300C030C300F003F
:1056D20000808000808080000020312E0E3120006A
:1056E200808080000080808080818E70180601009A
:1056F20000808080808080000021302C22213000B8
:1057020000000000807C020200000000003F4040D8
:1057120000000000FF00000000000000FF00000089
:105722000002027C800000000040403F00000000B8
:105732000006010102020404000000000000000053
:105742000000000000000000002F00000000070021
:10575200070000147F147F1400242A7F2A1200629B
:10576200640813230036495522500F090F0900001F
:1057720000001C224100000041221C000014083ECF
:1057820008140008083E0808000000A06000000895
:1057920008080808000060600000002010080402E9
:1057A200003E5149453E0000427F400000426151A7
:1057B2004946002141454B31001814127F10002741
:1057C20045454539003C4A49493000017109050304
:1057D20000364949493600064949291E0000363635
:1057E2000000000056360000000814224100001498
:1057F2001414141400004122140800020151090675
:1058020000324959513E007C1211127C007F4949F5
:105812004936003E41414122007F4141221C007F26
:1058220049494941007F09090901003E4149497A34
:10583200007F0808087F0000417F410000204041AE
:105842003F01007F08142241007F40404040007F1A
:10585200020C027F007F0408107F003E4141413E5E
:10586200007F09090906003E4151215E007F0919A6
:1058720029460046494949310001017F0101003FA3
:105882004040403F001F2040201F003F4038403F23
:105892000063140814630007087008070061514987
:1058A200454300007F41410000020408102000002F
:1058B20041417F0000040201020400404040404098
:1058C200000001020400002054545478007F484430
:1058D200443800384444442000384444487F003867
:1058E2005454541800087E0901020018A4A4A47C90
:1058F200007F080404780000447D4000004080845A
:105902007D00007F102844000000417F4000007CA1
:1059120004180478007C08040478003844444438AD
:1059220000FC242424180018242418FC007C0804F9
:10593200040800485454542000043F444020003CD2
:105942004040207C001C2040201C003C4030403C59
:10595200004428102844001CA0A0A07C00446454E9
:085962004C4414141414141435
:10596A002048617264773A202050494320436C6989
:10597A00636B65722031384634374A3533200D0A55
:10598A00204F6C6564205353443133303620313212
:10599A003878333220302E3936200D0A20445331DC
:1059AA00384232302073656E736F72200D0A2047B9
:1059BA0050532055426C6F7820374E200D0A2055DF
:0A59CA0041525432200D0A0D0A006C
:1059D40020536F75726365203A20436C69636B656D
:1059E400725F31384634374A35335F55415254314A
:1059F4005F4F6C65645F535344313330365F4453B7
:105A040031384232305F475053374E5F554152541C
:105A1400325F393630306264735F5F323032312D39
:095A2400303533312E630D0A0008
:105A2D0020446F73736965723A433A5C5F4D696BDD
:105A3D00726F435C5F4D657350726F6A6574735F0F
:105A4D004D696B726F435C5F31384634374A35337D
:105A5D005F4750535F55415254315F554152543257
:105A6D005F445331384232305F4F4C45440D0A008C
:105A7D0020417574726573203A20204F4C45445F68
:105A8D00493243325F3139303830312E63202C208A
:105A9D004F4C45445F4932435F3139303830312EF8
:105AAD0068202C204F4C45445F5461626C65735FD8
:0B5ABD00313930382E680D0A0D0A0048
:105AC80033206C69676E657320646520323020630B
:105AD800617273204142434445464748494A4B4C0A
:105AE8004D4E4F505152535455565758595A20619C
:105AF80062636465666768696A6B6C6D6E6F707106
:085B0800727374757677780062
:105B100020554152543120666F7220484331322063
:105B20006D617070656420393630302C382C4E2C05
:105B3000312054582070696E205244362D52503214
:105B400032202C2052782070696E205244352D521C
:065B50005032330D0A0083
:105B56002050726F6A65743A436C69636B65725F55
:105B660031384634374A35335F55415254315F4FE9
:105B76006C65645F445331384232305F4750533767
:105B86004E5F55415254325F323032312E6D637062
:055B960070690D0A001A
:025B9B00000008
:045B9D000000000004
:025BA1000600FC
:025BA300000000
:105BA500525C00A25D00D25D00325E00025E0072B2
:105BB5005D00B25C00825C00E25C00425D00125D4B
:015BC50000DF
:045BC60000000000DB
:0C5BCA002863007463006D630038630002
:025BD6000000CD
:015BD80000CC
:025BD9002C009E
:025BDB002C009C
:015BDD0000C7
:105BDE0020496E666F7320616666696368E9657356
:105BEE0020766961205541525431206D6F64756C79
:105BFE00E9657320656E20666F6E6374696F6E2043
:105C0E00646520425031206574204250320D0A00E6
:105C1E0020554152543220666F722047505320391E
:105C2E003630302C382C4E2C312054582070696E62
:105C3E0020524336202C2052782070696E20524319
:045C4E00370D0A0004
:105C52000080F0FCFEFE3F0F0F0F3FFEFEFCF080C7
:105C620000FFFFFFFFFF0000000000FFFFFFFFFF3C
:105C720000030F3F7F7FFCF0F0F0FC7F7F3F0F01BE
:105C8200001F1F1F1F1F1F1F1F9FFFFFFF3F1F0F11
:105C92000000000000E0F8FCFF7F0F03000000009E
:105CA200000000F0FFFFFFFF0700000000000000FF
:105CB2000080F0F8FCFE3E0F0F0F1F7F7E7E7C708F
:105CC20000FFFFFFFFFF3C1E1E1E3EFEFCFCF0E03D
:105CD20000010F3F7F7FF8F0F0F0F8FF7F3F1F07D2
:105CE20000F0FCFEFEFF1F0F0F0F1FFFFEFEFCF079
:105CF2000081C3E7FFFF7E3C3C3C7EFFFFE7C381A0
:105D0200000F3F7F7FFFF8F0F0F0F8FF7F7F3F0F3B
:105D12000000000000000000000000000000000081
:105D22000000000000000000000000000000000071
:105D320000000000000000000000FFFFFFFF000065
:105D420000E0F8FCFEFF1F0F0F0F1FFEFEFCF080AD
:105D520000070F3F3F7F7C7878783CFFFFFFFFFF13
:105D6200000E3E7E7EFEF8F0F0F07C7F3F1F0F01BA
:105D7200000080FCFFFFFF3F1F1F1F1F1F1F1F0090
:105D820000183F3F3F3F1F0F0F0F1FFFFEFEF8E0BF
:105D920000061F3F7F7FFCF0F0F0F87F7F3F1F0778
:105DA200000000C0E0E0F0F87CFEFFFFFFFF000013
:105DB200000000030101000000FFFFFFFFFF0000E1
:105DC200000000000000000000FFFFFFFFFF0000D6
:105DD20000E0F8FCFEFE1F0F0F0F1FFFFEFEFCF09F
:105DE200000000000080C0E0F0F8FE7F3F1F0701C6
:105DF20000C0F8FCFFFFFFFFF9F9F8F8F8F8F8F82F
:105E02000000000000C0E0F8FCFFFFFFFFFF000001
:105E1200C0E0F8FCFFBF8F8381FFFFFFFFFF8080A0
:105E2200070707070707070707FFFFFFFFFF070728
:105E32000030787E7E7F1F0F0F1FFFFEFEFCF000FA
:105E4200000000000000000E0E0F1FFBFBF9F0C067
:105E520000061F3F7F7FFCF0F0F0FC7F7F3F1F07B3
:105E6200205265637520646520484331322064699D
:105E72007374616E74202855415254312052582057
:0D5E8200E020393630307329203A0D0A0037
:105E8F002070696E20524234206F757470757420C3
:105E9F003D3E206364652053455420286D6F646533
:0C5EAF002041542920484331320D0A00E4
:105EBB00204275732049324320706F757220456301
:105ECB0072616E204F4C454420535344313330366E
:0A5EDB00203132387833320D0A000E
:105EE500205265746F7572204D61707061676573BE
:105EF5002070696E732055415254312065742055C8
:085F050041525432203D2000FE
:105F0D00205465737420536F6E6465204F57532072
:105F1D004453313842323020737572205241322051
:035F2D000D0A005A
:105F30000D0A4B6579626F61726420546F756368F6
:105F4000205541525431206F722054696D656F7530
:035F5000742000BA
:105F53002042414420526563657074696F6E206FFF
:105F630075204465636F64616765204747410D0A87
:015F7300002D
:105F7400526563657074696F6E2073757220554144
:105F8400525432205258203D20475053203A0D0A93
:015F9400000C
:105F9500206F752034206C69676E657320646520F9
:105FA500323020636172732036783870200D0A0014
:105FB5002055415254322C2077616974696E6720EF
:0D5FC500475053206461746173203A20003E
:105FD200204D435520203A2031384634374A353354
:0D5FE2005F51464E5F343470696E0D0A0049
:105FEF0020524431202D2D3E2049324332202D2D79
:0D5FFF003E534441204F4C4544200D0A0004
:10600C0020524430202D2D3E2049324332202D3E4B
:0C601C002053434C204F4C45440D0A001B
:10602800205265746F7572206465204843313220B0
:0A6038006C6F63616C203A0D0A00E2
:10604200204D617576616973652052656365707470
:0A605200696F6E204750530D0A00DD
:10605C00205265746F75722064652048433132207C
:0A606C006C6F63616C203A0D0A00AE
:106076002041666669636865203320636172732018
:09608600537065636961757800CF
:10608F00204F4C4544204C4344204E6F6E20747279
:08609F006F7576E9200D0A007F
:1060A70020496E69742055415254312039363030B9
:0660B7006264730D0A0093
:1060BD00204C6174693A20202020202020202020AF
:0660CD002020202020002D
:1060D30020416C74693A2020202020202020202099
:0660E30020202020200017
:1060E9004932433220696E6974206174203130303D
:0660F9004B687A0D0A005D
:1060FF00204C6F6E673A2020202020202020202067
:06610F00202020202000EA
:1061150020506F77657220737570706C793A2034F2
:066125002E35560D0A00A4
:10612B0020323020436861727320737572204C6982
:06613B00676E65203100D3
:10614100426967204D7367206465203630206361A2
:066151007273203A2000E9
:1061570020426F75636C652023202020202020209B
:056167002020202000B3
:10616C004C34204E554D424552532030313233344D
:05617C00353637380044
:106181003132333435362D4142432D6162632D3630
:05619100373839300031
:106196002037202042696720436172732020313600
:0561A6007831362000F5
:1061AB0031323334353637383930313233343536A2
:0561BB00373839300007
:1061C000204F6C65642046494C4C207769746820E8
:0561D000307846460096
:1061D5004D73672031342063617273207461696C7B
:0561E5006C6520320092
:1061EA004D7367207375722034656D204C69676E34
:0461FA0065202000FC
:1061FE002054656D7065723D20202020202020B037
:02620E0043004B
:10621000204D657375726520445331384232303DEC
:0262200020005C
:10622200436865636B20446576696365204020009E
:1062320030313233343536373839414243444546BA
:106242002046616D696C7920436F6465203A2000B5
:0F62520020436F6E66696720484331320D0A00A2
:0F62610020436F6E66696720484331320D0A0093
:0F6270000D0A204F4C454420696E69740D0A00D9
:0E627F00206973206E6F7420666F756E640068
:0D628D002078203130306D7365630D0A00FC
:0D629A00204F4C454420696E69740D0A00C8
:0C62A7002020202020416C74203A2000B0
:0C62B3002020202048444F50203A2000BA
:0B62BF00204F4C4544204F4E0D0A00BC
:0B62CA00202E2E42414420210D0A002E
:0B62D500202020536174656C3A20000B
:0A62E000202020204669783A2000B3
:0A62EA0020666F756E64204F4B00B4
:0962F400322020484152445700B9
:0962FD0020204C6174203A2000BD
:096306002041542B52580D0A00ED
:09630F002041542B52580D0A00E4
:0863180020204352433D200008
:0863200020494431203D20001A
:0863280000007E66667E0000A5
:086330002E2E204F4B0D0A0038
:086338000F090F000000000036
:08634000206F6E20493243007A
:08634800204C6F6E203A20008A
:08635000202E2E4F4B0D0A0018
:076358004B4D4C203A2000E0
:07635F0024475047474100AD
:076366003132342E393600FC
:07636D00060C1C7C1C0C0651
:07637400C030383E383060F4
:06637B002041540D0A0050
:066381002041540D0A004A
:05638700302E30300053
:05638C00302E3030004E
:05639100B043202000D4
:05639600302E30300044
:04639B00205A200064
:04639F002059200061
:0463A300205820005E
:020000040001F9
:08FFF800ACF7FCFFFFFBFFFB6F
:00000001FF
